:10617000011300000B01013C0200000301FA0400BE
:10618000FA0500030A0A5A0B001E0C00FA0D000360
:106190000E00030F0164100096120132130AFA1464
:1061A000010215010217010A1801FA1905321A0134
:1061B0000A1B01FA1C05321FFFFF20FFFF23011EEF
:1061C0002400642A00FA2B00FA2C50782D003C2E73
:1061D00000462F001E3000643250783432FA350108
:1061E00064360164370150380A643C00643E003C68
:1061F0003F000140FFFF411450420A5A430AC8447D
:1062000005324500B44600FA47013C4803034C0000
:10621000FA4EFFFF500303510596520A32530B46C4
:10622000540A96560103570546580002590A465A21
:1062300032FA5B010A5C0A325E000A5F00FE61FF0F
:10624000FF64010F6600026701016A0A3C6B0000EF
:106250006C32967300007400007801327901327E4E
:10626000FFFF81FFFF84FFFF8500AF8600018700ED
:10627000FA89010A8A00009900009D0A969E000191
:106280009FFFFFFAFAFA00000B01013C0200000335
:1062900001FA0400FA0500030A0A5A0B001E0C005A
:1062A000FA0D00030E00030F016410009612013274
:1062B000130AFA14010215010217010A1801FA194A
:1062C00005321A010A1B01FA1C05321FFFFF20FFCD
:1062D000FF23011E2400642A00FA2B00FA2C5078B8
:1062E0002D003C2E00462F001E30006432507834C2
:1062F00032FA350164360164370150380A643C00D3
:10630000643E003C3F000140FFFF411450420A5AE6
:10631000430AC84405324500B44600FA47013C48E8
:1063200003034C00FA4EFFFF500303510596520A37
:1063300032530B46540A9656010157054658000140
:10634000590A465A32FA5B010A5C0A325E000A5F59
:1063500000FE61FFFF64010F6600026701016A0A27
:106360003C6B00006C3296730000740000780132C0
:106370007901327EFFFF81FFFF84FFFF85FFFF86EB
:10638000FFFF87FFFF8901028A00009900009D0A34
:10639000969E00019FFFFFFAFAFA0065006F0079F0
:1063A0000083008D009700A100AC00B600C000CAB9
:1063B00000D400DE00E800F2005B0063006A0072B7
:1063C000007A008200890091009900A100A800B025
:1063D00000B800BF00C700CF00D600DF00E600EE27
:1063E00000F600400046004C00520059005F006576
:1063F000006B00710077007D00830089008F00959D
:10640000009C00A200A800AE00B400BA00C000C604
:0E64100000CC00D200D900DF00E500EB00F167
:1035E700900054E0D3940440149007C5E0FEA3E094
:1035F700FF906172126557E493F59980129007C5A1
:10360700E0FEA3E0FF906286126557E493F5999078
:1036170007C5E0FEA3E0FF906170E493FC7401939B
:10362700FDEFB50507EEB50403754D009007C5120C
:10363700653E2275A71085F97285FA737E017F00B2
:10364700E573126530E5722FFF50010E8E598F5AC0
:10365700900017E0FCA3E0FDEF2DFDEE3CFC8C5B3A
:103667008D5C2275A71085F97285FA737E017F003C
:10367700E573126530E5722FFF50010E8E598F5A90
:103687009000E7E0B40210AC2CAD2DEF2DFDEE3C21
:10369700FC8C5B8D5C8016AE59AF5A900017E0FC2E
:1036A700A3E0FDEF2DFDEE3CFC8C5B8D5C22AE595B
:1036B700AF5A740C8E048F05FF1265208C5B8D5CEE
:1036C700AE59AF5A740C8E048F05FF12654B8C5997
:1036D7008D5AE55A45596013740CC3955AFFE49502
:1036E70059FE8E598F5A785B126584E572A85BB8CC
:1036F7000015D3955C4010E572C3955CFFE4955BBC
:10370700FE8E5B8F5C8010E572243CC3955CFFE402
:10371700955BFE8E5B8F5C757200AE5BAF5C74135E
:103727006F4E600674146F4E7018AE5BAF5C741307
:103737006F4E70057572018003757202755C1275A4
:103747005B00AE5BAF5C74276F4E600674286F4EEC
:103757007018AE5BAF5C74276F4E70057572018091
:1037670003757202755C26755B00AE5BAF5C743BDC
:103777006F4E6006743C6F4E7018AE5BAF5C743B67
:103787006F4E70057572018003757202755C3A752C
:103797005B0022900095E0B40104C2108002D210B1
:1037A700900096E0B40104C2118002D2119000D3B8
:1037B700E075F0DCA4FFAEF0740A8E048F05FF12EB
:1037C70065209007BBECF0A3EDF0A20D4016740343
:1037D7008C068D0712653074011200399007B9EE17
:1037E700F0A3EFF07E017F00900091E0126530902A
:1037F70000D4E08E048F05FF126520740AFF12655E
:10380700208D5F9000DDE075F0DCA4FFAEF0740A58
:103817008E048F05FF1265209007BFECF0A3EDF033
:103827009000DFE060139000DFE0F5F0741684FF8E
:103837007E00EF9007C9F0800674649007C9F09086
:1038470000D5E0900079F090011FE0900063F090C0
:1038570000AEE0900065F0900083E0900067F09084
:103867000109E090006CF074E3900078F09000BEDE
:10387700E0B40B0874E3900078F0805A9000BEE043
:10388700B419129000D4E090638512008CE49390F1
:103897000078F080419000BEE0B41E129000D4E0A2
:1038A7009063A312008CE493900078F08028900036
:1038B700BEE0B428129000D4E09063CD12008CE4EF
:1038C70093900078F0800F9000BEE0B44608900017
:1038D700B5E0900078F090007DE0FE9000D7E0B56D
:1038E700063390007CE0FE9000BBE0B50627900011
:1038F7007FE0FE9000D9E0B5061B90007EE0FE90C9
:1039070000E7E0B5060F900080E0FE90008EE06EC5
:103917007003023A729000E7E06008740790010AAA
:10392700F08006740A90010AF09000D7E0B402060E
:1039370074039000D7F090008EE0B40106740090F5
:1039470000F4F090008EE0B4020674009000D9F005
:1039570090008EE0B4030674009000E6F09000BB80
:10396700E0601474189000A2F074009006CFF07411
:10397700009006D0F0800C74009000A2F0741890AC
:1039870006CFF09000D9E0D3940140147419900148
:103997000CF074009006D3F074009006D4F0800CFD
:1039A700740090010CF074199006D3F09000BBE0FE
:1039B700B40214741A9000A3F074009006D7F07440
:1039C700009006D8F0800C74009000A3F0741A9051
:1039D70006D7F09000E7E0701474049006E3F074E3
:1039E700059006E7F074069006EBF08024740090CB
:1039F70006E3F074009006E4F074009006E7F074B4
:103A0700009006E8F074009006EBF074009006EC66
:103A1700F0D2289000D7E090007DF09000BBE090B6
:103A2700007CF09000E7E090007EF09000D9E090F5
:103A3700007FF090008EE0900080F090008EE09084
:103A47000064F09000D7E0900066F09000C9E09025
:103A57000068F09000E7E0900069F09000BBE0900C
:103A6700006AF09000D9E090006BF09000F1E0B4AC
:103A77000117900023740FF0A374FFF0900025E462
:103A8700F0A3F074029000F1F09000F1E0B403416C
:103A9700900025E0FEA3E0FF900023E0FCA3E0FDFB
:103AA70012657C74101265307408120039EF9000AB
:103AB70075F0EF700674FF900075F074009000F1D8
:103AC700F0900024E0900076F0900023E0900077DB
:103AD700F0900082E0900043F0900043E0241490BF
:103AE7000044F0900043E02428900045F090004403
:103AF700E0D3943C400B900044E0C3943C900044D6
:103B0700F0900045E0D3943C400B900045E0C3940F
:103B17003C900045F0900049E4F0900043E06413C6
:103B27006007900043E0B41420900043E0B413060C
:103B37007402900049F0900043E0B41406900049E5
:103B47007401F07415900043F0900043E06427601F
:103B570007900043E0B42820900043E0B4270674A0
:103B670002900049F0900043E0B4280690004974A1
:103B770001F07429900043F0900043E0643B600734
:103B8700900043E0B43C20900043E0B43B0674024D
:103B9700900049F0900043E0B43C0690004974015E
:103BA700F09000437401F090004AE4F0900044E084
:103BB70064136007900044E0B41420900044E0B41C
:103BC7001306740290004AF0900044E0B414069083
:103BD700004A7401F07415900044F0900044E064CA
:103BE700276007900044E0B42820900044E0B42701
:103BF70006740290004AF0900044E0B42806900052
:103C07004A7401F07429900044F0900044E0643B4A
:103C17006007900044E0B43C20900044E0B43B06C9
:103C2700740290004AF0900044E0B43C0690004AC9
:103C37007401F09000447401F090004BE4F09000A0
:103C470045E064136007900045E0B41420900045F8
:103C5700E0B41306740290004BF0900045E0B414F2
:103C67000690004B7401F07415900045F0900045E4
:103C7700E064276007900045E0B42820900045E005
:103C8700B42706740290004BF0900045E0B4280674
:103C970090004B7401F07429900045F0900045E0C6
:103CA700643B6007900045E0B43C20900045E0B4D9
:103CB7003B06740290004BF0900045E0B43C069040
:103CC700004B7401F09000457401F0900082E0FE13
:103CD7009000E5E02E90004DF09000C0E0B4013771
:103CE70090004DE075F00F84AFF07E00EF90004D2F
:103CF700F0EFB40A06740B90004DF090004DE0B45D
:103D07000906740890004DF090004DE0240F9000D4
:103D17004EF075500F802B90004DE075F00A84AF80
:103D2700F07E00EF90004DF0EFB40A0690004D745E
:103D370001F090004DE0B40906740890004DF0754D
:103D4700500A9000C8E0900046F0900046E06414E6
:103D5700600F900046E064286007900046E0B43C9E
:103D670006900046E004F0900046E06413600F9070
:103D77000046E064276007900046E0B43B069000E9
:103D870046E014F0900046E0D3943C400B90004688
:103D9700E0C3943C900046F0900046E02414900065
:103DA70047F0900046E02428900048F0900047E054
:103DB700D3943C400B900047E0C3943C900047F0FD
:103DC700900048E0D3943C400B900048E0C3943CFB
:103DD700900048F022C293C294C291C292C287C295
:103DE70090E5B554EFF5B5E5B554DFF5B5C296C224
:103DF70095C2A0C297C2A2C2A1E5B554BFF5B5E569
:103E0700B5547FF5B5E5B554FBF5B5C213755D46F9
:103E17009000CBE07005756C028003756C037554D8
:103E27000075530090000C74FFF0A374DCF0C21906
:103E3700C21BC21D74C8900037F074C890003BF0D5
:103E470074C890003FF0755200755100C20D754659
:103E570000E56EB40903756E00756200900019E401
:103E6700F0A3F0756F10C216C217C2189007BBE017
:103E7700FEA3E0FF74031265307401120039900746
:103E8700B9EEF0A3EFF0C202755600755500900029
:103E970010E4F0A3F0C22975580075570090008D03
:103EA700E075F032A4FDACF0900021ECF0A3EDF04A
:103EB700C239C2122275A71085F97285FA737E017D
:103EC7007F00E573126530E5722FFF50010E8E59A2
:103ED7008F5AAC5BAD5CEF2DFDEE3CFC8C5B8D5CD3
:103EE700D293D294D291E55CF5FBE55BF5FCE55CFA
:103EF700F5E9E55BF5EAE55CF5EBE55BF5EC75A760
:103F0700002285F97285FA737E017F00E5731265D9
:103F170030E5722FFF50010E8E598F5A7E017F7642
:103F2700900106E0126530AC59AD5AED2FFFEC3E1B
:103F3700FE8E5B8F5CE55CF5EDE55BF5EE90007959
:103F4700E4F07412900050F02285F97285FA737EBE
:103F5700017F00E573126530E5722FFF50010E8E69
:103F6700598F5A9007BBE0FCA3E0FDEF2DFDEE3C17
:103F7700FC8C5B8D5CE55CF5FDE55BF5FE2205637E
:103F870022A2DBB340089000D5E0900079F0A2DCD4
:103F9700B34006C296C295C2A075D8402285A771C4
:103FA70075A7109000E7E0B4011DA2D8B34004C282
:103FB70093C292A2D9B34004C294C287A2DAB34093
:103FC70004C291C2908031A2D8B34002C293A2D951
:103FD700B34002C294A2DAB34002C2919000E7E074
:103FE700B40215A2DBB34002C292A2DCB34002C204
:103FF70087A2DDB34002C29075D8408571A7229091
:104007000047E4936406600280FE74C89007C1F815
:10401700E4F0E8A3F075B50075840175A70075FF96
:10402700A090004CE4F075C91075A70F75A1C7756E
:10403700A70075D90075CE0C75A70F75F1FE75F23F
:10404700FF75F30775F47875A4BA75A5FF75A6070C
:1040570075AE0075AFFF75D48175D5FF75D6FF7541
:10406700D7FF75A70075A20175A14775F80975D81F
:104077000075D90475DD0975DE0975D84075A71077
:1040870075D80075D90475DA0975DB0975DC09750A
:10409700DD0975DE0975DF0975D84075A70075E676
:1040A7000875E71075BC0175BE0475BD6C75BE0754
:1040B70075BDA075BE0875BD0175BC0075BB1875CB
:1040C700BC2075BA0875E88075D11375A70F75E11F
:1040D7000575E20075C740123DDC7597007597803E
:1040E700740A1265107597C0E5975420700280F81E
:1040F700758F0275A700D2AF75980075A90C75A7C3
:104107000F75AB4375ADFB75AC1E75A71075C91858
:1041170075CA0075CB0075C80475A7007589127537
:104127008E04758C00758A00C2A9D28C758D0075B6
:104137008B00D2ABD28E75EF0675D944C29974C87D
:10414700F5097508001200E375B5001204E37463FE
:104157009007C1F8E4F0E8A3F012036F74C8900762
:10416700C1F8E4F0E8A3F07464F5097508001200DB
:10417700E3900064E090008EF0C22190008EE0D3BF
:1041870094034006740090008EF090008EE0905DDE
:1041970085F82828738028A2B44002D22180207590
:1041A700A70F75F30F75A700A2A34002D221800FB6
:0F41B70075A70F75F31775A700A2A44002D221B8
:0C5D850002419C02419E0241A60241B76F
:1041C600A221B34066757208E572D3940E5020E5BD
:1041D600729007C1F8E4F0E8A3F012023E7464F5A9
:1041E600097508001200E37872740126F650D97436
:1041F600029000CAF090008EE0D39403400674004B
:1042060090008EF090008EE0905D91F828287380E3
:104216001674009000F4F0800E74009000D9F080BF
:074226000674009000E6F0B1
:0C5D910002421502421702421F02422784
:10422D00D2208064757201E572D394075020E57237
:10423D009007C1F8E4F0E8A3F012023E7464F509AA
:10424D007508001200E37872740126F650D97401D6
:10425D009000CAF090008EE0D39403400674009055
:10426D00008EF090008EE0905D9DF82828738016EA
:10427D0074009000F4F0800E74009000D9F0800668
:06428D0074009000E6F051
:0C5D9D0002427B02427D02428502428DE0
:10429300C220900063E090011FF0900064E0900062
:1042A3008EF0900065E09000AEF0900066E0900024
:1042B300D7F0900067E0900083F0900068E09000F2
:1042C300C9F0900069E09000E7F090006AE0900088
:1042D300BBF090006BE09000D9F090006CE090018F
:1042E30009F09000D4E07006740A9000D4F09000B6
:1042F300B5E0700674E39000B5F09000BBE0049065
:10430300007CF012379AE5B54401F5B574069000C8
:1043130052F07401900053F07403900055F074054B
:10432300900056F0745A900057F07405900058F0BE
:10433300900054E0B404067404900058F0740090A4
:104343000059F0740090005EF0740090005FF07408
:1043530001900060F07400900061F074FF900062BF
:10436300F07436900158F07430900159F0742D9028
:10437300015AF0743690015BF0742B90015CF07479
:104383004890015DF0746F90015EF0746D90015F71
:10439300F07465900160F07420900161F0742090D6
:1043A3000162F07433900163F07443900164F0741C
:1043B30079900165F0746C900166F09000F0E090E4
:1043C3000075F09000A7E0900076F09000A8E090D0
:1043D3000077F0A2B6B3920EA2B3B3920FA2A4B326
:1043E3009225A2B4B39226A2A3B39227900071E4BC
:1043F300F0756E00743A900781F074FD900782F0B7
:10440300900072E4F09007BBE0FEA3E0FF74031298
:10441300653074011200399007B9EEF0A3EFF0751F
:104423006D01900050E4F0C224756200C214D215ED
:10443300C202757000C22BD203C22CD204C22DD289
:1044430005C22ED206C22FD207C230D208C231D241
:1044530009C232D20AC233D20BC234D20CC222C234
:1044630023C22812009E755E00756A007560007590
:104473006432756500756600756700756800756957
:1044830000900019E4F0A3F0756B00D2B2D2A4D26D
:10449300B0D2B1D2A3D2A7D2A6D2A5D2B790008D63
:1044A300E0D394FA400674FA90008DF07E017F0009
:1044B300900077E0126530900076E02FFF50010EF8
:1044C300900023EEF0A3EFF0EFD394FFEE940F40B0
:1044D30007900023E4F0A3F0900075E0700674FFEA
:1044E300900075F074009000B4F09000CAE0D3948B
:1044F30002400674019000CAF09000CBE07005758D
:104503006C028003756C039000CCE0D394014006E9
:1045130074009000CCF09000D2E0C3940A5006746B
:104523000A9000D2F09000DCE0700674019000DC89
:10453300F09000DCE0B4FF0674FE9000DCF0900025
:10454300E3E0D394FE400674FE9000E3F09001098B
:10455300E0D3940240067401900109F090011FE03A
:10456300D394014006740190011FF074019000E997
:10457300F074019000EAF074009000F1F074009080
:10458300010DF07400900111F074299006C7F074C6
:104593002A9006CBF0741B9006DBF0741C9006DFA8
:1045A300F0D29C9000BCE0D39404400674049000C5
:1045B300BCF09000EEE0D39404400674049000EE47
:1045C300F0E56FD394104003756F109006C8E0D3E5
:1045D300940C400674009006C8F09006CCE0D39487
:1045E3000C400674009006CCF09006D0E0D3940CF7
:1045F300400674009006D0F09006D4E0D3940C40AB
:104603000674009006D4F09006D8E0D3940C4006CC
:1046130074009006D8F09006DCE0D3940C40067446
:10462300009006DCF09006E0E0D3940C40067400A2
:104633009006E0F09006E4E0D3940C4006740090FA
:1046430006E4F09006E8E0D3940C4006740090066C
:10465300E8F09006ECE0D3940C400674009006EC6E
:10466300F0D2EC75CF01A298B34005C2981206169A
:10467300E54D6006A299B3B340028005C299120AC0
:10468300B4E54E64016005E54EB4040280D5C28EE4
:104693007E107F00E563126530E58D75F010A4FD93
:1046A300ACF0EF2DFDEE3CFCE58B75F01084FF7E46
:1046B30000ED2FFFEC3EFE8E538F54D28E9000AE52
:1046C300E060099000AEE0C3943D4002805C90003E
:1046D3001B12653E90001BE0FEA3E0FF90001DE06F
:1046E300FCA3E0FDEFB50542EEB5043EB21FA20DFB
:1046F300B3401975E700A21FB34008E5B54404F5BC
:10470300B58006E5B554FBF5B575E71090001DE0DF
:10471300FEA3E0FF90001FE0FCA3E0FDEF2DFDEE04
:104723003CFC90001DECF0A3EDF09000BBE06009B1
:104733009000BBE0C394034002806F1229C0A20D16
:10474300B35009900071E0C39423400280069000A7
:10475300A5E0F545E54575F005A4FFAEF09007C368
:10476300EEF0A3EFF0900092E0C395604007E55EA2
:10477300C3955F50079007C3E4F0A3F0AE2EAF2FAD
:104783009007C3E0FCA3E0FDEFD39DEE9C4004C281
:10479300A1800B900071E0C394325002D2A190002B
:1047A300BBE0B40205A2A1B392A29000BBE0B403A4
:1047B3001C122ADBAE2EAF2F9007C3E0FCA3E0FD53
:1047C300EFD39DEE9C4004D2A18002C2A19000963B
:1047D300E06009A2B3300F01B3B340028029A2B352
:1047E300300F01B34021A2B3301101B3400CA21327
:1047F300B34002D212A211B3920FA211B330B3018C
:10480300B34004A211920FA2B6300E01B3500302BB
:104813004E81A2B6300E01B35003024E81A2B630D0
:104823001001B35003024CC5756D00055DA213B3AF
:10483300B35013AE53AF5490000CE0FCA3E0FDED76
:10484300C39FEC9E4003024971E55D64136005E577
:104853005DB42709E55D2402F55D02494DE56CB4BD
:10486300032EA229B34022E55DB43B03756C01E539
:104873005DC3943B50069000507401F0E55DD39402
:104883003B40067402900050F0755D01D229805CB4
:10489300E56CB40206756C01755D3BE55DB43B05E3
:1048A300755D018047900050E07032E55DC3943B35
:1048B30050069000507401F0E55DD3943B400674BC
:1048C30002900050F0E55DC3943B5002D224E55DB5
:1048D300D3943B4002D224C296C295C2A09000CB8F
:1048E300E0B40105123DDC8003755D01A212B34003
:1048F30005755D01C2129000AEE060099000AEE064
:10490300C3943D4002804390001BE0FEA3E0FF9070
:1049130000AEE08E048F05FF12652074018C068DB6
:104923000712003990001FEEF0A3EFF090001FE094
:10493300F8A3E090001DC8F0A3C8F090001BE4F0BA
:10494300A3F0C21FE5B554FBF5B5AE55AF56AC5356
:10495300AD54EF2DFDEE3CFC74028C068D07120066
:10496300398E558F56A224B34002C224803AAE55E5
:10497300AF56AC53AD54EF2DFDEE3CFC74018C06E9
:104983008D071200398E558F56E56CC39402500D76
:10499300AC53AD547418C39D74159C400280091226
:1049A3003DDC7406900050F0E55DB43B1274039057
:1049B3000050F0D2249000CBE0B40103123DDCAEF2
:1049C30057AF58AC53AD54EF2DFDEE3CFC8C578DD7
:1049D30058AE53AF54EFD39DEE9C4011900013E0BB
:1049E300FAA3E0FBEBC394E8EA9403400280069049
:1049F300001312653E900010E0FEA3E0FFAC53AD40
:104A030054EF2DFDEE3CFC900010ECF0A3EDF09084
:104A130000CBE0B40118AE53AF5474051265307483
:104A23000112003990000CEEF0A3EFF08011AE53A9
:104A3300AF54740212653090000CEEF0A3EFF0C295
:104A43008E758D00758B0075630075540175530069
:104A5300D28EE55D240975F00A84AFF07E00EF4E37
:104A63007075900010E0F8A3E090000EC8F0A3C8A2
:104A7300F090000EE0FEA3E0FFEF4E600B7CA97DFB
:104A8300B712641E8E518F52900010E4F0A3F0AE63
:104A930051AF527428BE00039F5010E5622FFF50A0
:104AA300010E74011200398E518F528552629000AB
:104AB300D2E0A851B8000DD395524008E5529000BA
:104AC3004FF080099000D2E01490004FF0E56C6045
:104AD30006755200755100E55D64096005E55DB436
:104AE30018099000BBE0600312202B9000C0E0B4D3
:104AF300012F90004DE0655D600990004DE0241E9C
:104B0300B55D08756E00855D50801490004EE065BC
:104B13005D600990004EE0241EB55D03756E008054
:104B23004390004DE0655D600990004DE0241EB5A3
:104B33005D08756E00855D50802A90004DE0240A63
:104B4300655D601D90004DE02414655D6013900069
:104B53004DE02428655D600990004DE02432B55D89
:104B630003756E00A214B35006A213B3B34003023D
:104B73004C1A900087E0B40173900109E0B4021469
:104B8300120C5590007AE075F0BEA4FFAEF08E5B78
:104B93008F5C8056E56675F00A84FF7E0090058180
:104BA300126557E0F55A755900AE59AF5A9000ACEB
:104BB300E012653074648E048F05FF1265208C5BF0
:104BC3008D5CE55C900012F0AE59AF5A900085E021
:104BD30012653074648E048F05FF12652074BE8CD9
:104BE300068D071265308E5B8F5C8017900085E021
:104BF30075F0BEA4FFAEF08E5B8F5C9000ACE090CE
:104C03000012F0E560C394CC5006900085E070027A
:104C13008003123EBCD214E56CB40106E55D640961
:104C230060028009756F019000517401F0E56C60BA
:104C330003024CC09000CEE0600D900079E0A851D3
:104C4300B800069552400280409000CEE0B4021FA7
:104C5300900043E0655D600F900044E0655D600790
:104C6300900045E0B55D03756F03756B00800CC262
:104C730000756B00900019E4F0A3F0900079E060F8
:104C8300067409900050F08034900043E0B55D0B4A
:104C9300756F019000517401F08022900044E0B5DB
:104CA3005D0B756F017402900051F0801090004508
:104CB300E0B55D09756F017403900051F0A210B364
:104CC300920EA210B330B601B35003024E81756D3C
:104CD30001E5B54401F5B57423900071F0A210927B
:104CE3000EE55DD3944A4014D213E55DD39480401E
:104CF3000B7403900050F0D224755D469000D6E00B
:104D0300B40107E569C3941440028009123DDC74C1
:104D130013900050F0A22B300301B3501D75E70030
:104D2300A22BB34008E5B54408F5B58006E5B554B4
:104D3300F7F5B575E710A22B9203A22C300401B34B
:104D4300501D75E700A22CB34008E5B54402F5B544
:104D53008006E5B554FDF5B575E710A22C9204A2C3
:104D63002D300501B3500FA22DB34004D29780021A
:104D7300C297A22D9205A22E300601B3500FA22E88
:104D8300B34004D2A28002C2A2A22E9206A22F3066
:104D93000701B3500FA22FB34004D2A18002C2A1D6
:104DA300A22F9207A230300801B3501D75E700A26D
:104DB30030B34008E5B54440F5B58006E5B554BFCA
:104DC300F5B575E710A2309208A231300901B3504E
:104DD3001D75E700A231B34008E5B54480F5B58001
:104DE30006E5B5547FF5B575E710A2319209A232F5
:104DF300300A01B3500FA232B34004D2928002C2F0
:104E030092A232920AA233300B01B3500FA233B3F2
:104E13004004D2878002C287A233920BA234300CA3
:104E230001B3500FA234B34004D2908002C290A2C7
:104E330034920CE569C394415009740E900050F00C
:104E4300123DDC900058E0FE900054E004C39E4005
:104E530009900054E0D39406400974FB900050F08D
:104E6300123DDC90005DE0601590005DE0FE900077
:104E730057E06E600974FE900050F0123DDCA224EE
:104E8300B34006C296C295C2A0900106E0600CAE84
:104E930051AF527414BE00059F4002804890008EAB
:104EA300E0905DA9F8282873803BA2B4B35005A213
:104EB30026B340028005123F09D2268028A2A3B35D
:104EC3005005A227B340028005123F09D22780155F
:104ED300A2A4B35005A225B340028005123F09D214
:054EE3002580028000A3
:105DA900024EAB024EAD024EC0024ED3024EE60287
:025DB9004EE8B2
:104EE800A216B3B35008900046E0655D60028041A9
:104EF800A201B35006A200B3B34002802E12363A84
:104F0800E55CF5FBE55BF5FC75A700D293A202B35F
:104F18004002D2929000E7E0B4021012366AE55CD3
:104F2800F5EDE55BF5EE75A700D292C216D217D261
:104F380018A217B3B35008900047E0655D6002807F
:104F480041A201B35006A200B3B34002802E12362C
:104F58003AE55CF5E9E55BF5EA75A700D294A202AB
:104F6800B34002D2879000E7E0B4021012366AE537
:104F78005CF5FDE55BF5FE75A700D287D216C21772
:104F8800D218A218B3B35008900048E0655D6002DB
:104F98008041A201B35006A200B3B34002802E1292
:104FA800363AE55CF5EBE55BF5EC75A700D291A226
:104FB80002B34002D2909000E7E0B4021012366AC1
:104FC800E55CF5CEE55BF5CF75A700D290D216D299
:104FD80017C218E56F905DBBF828287302553A9000
:034FE80000EEE0F8
:065DBB00024FE4024FE775
:104FEB00905DEEF8282873121B078012121B0780A6
:0E4FFB000D121B918008121C3D8003121C3DFC
:0F5DEE00024FF2024FF7024FFC02500102500623
:10500900756F0202553A121D69121E80A239B3400A
:10501900229000B0E0F56B900081E0256BFE9000D6
:105029004FE075F01E84FC7F00EE2CF5347410906F
:105039000050F09007B9E0FEA3E0FF740A12653052
:1050490090000EE0FCA3E0FD740C8F02FF126520B6
:105059008D078C038E048A058B0612641E9007BD8A
:10506900EEF0A3EFF09000D7E0B401087478BE0029
:10507900059F4002800D74789007BDF8E4F0E8A31D
:10508900F0801B9007BDE0FEA3E0FF74F0BE0003B3
:105099009F500B74F09007BDF8E4F0E8A3F0E534F5
:1050A90070037534019007BDE0FEA3E0FFE5342FDE
:1050B900FF50010E9007BDEEF0A3EFF0756F03905E
:0350C9000051E0B3
:035DC10002500F7E
:1050CC00905DFDF82828738019A23A4003756F0A89
:1050DC008010A23A4003756F0B8007A23A4003750B
:0250EC006F0C47
:0C5DFD000250D30250D50250DE0250E7E5
:1050EE0002553A9006C8E06003122114900107E0C1
:1050FE00B40114900108E0A851B80004955250076D
:10510E00E55EC3955F4002800302519B9000BCE0B8
:10511E00D39402403F900090E02403A851B80004BD
:10512E0095525009900092E0D3956050028008D2BB
:10513E00017408900050F0900090E0A851B800055E
:10514E00D39552500B900092E02403C39560500209
:10515E00C2018039900090E02403A851B800049554
:10516E00525007E55EC3955F40028008D201740875
:10517E00900050F0900090E0A851B80005D39552E1
:10518E005009E55F240FC3955E5002C2019000D610
:10519E00E07007E569C3941440028002D201A201B7
:1051AE004005756F04800A756F10900019E4F0A326
:1051BE00F0A20DB34029E56675F00A84FF7E0090DB
:1051CE000581126557E0C394695005122060800F67
:1051DE009007BBE0F8A3E09007B9C8F0A3C8F002AF
:0651EE00553A9000BCE000
:065DC4000250F10251F053
:1051F400905E09F8282873120D3F8012120D3F802B
:0E5204000D120EED8008120F9F8003120F9FF7
:0F5E09000251FB02520002520502520A02520FCE
:105212009006CCE060031221F0756F0502553A1238
:1052220010AB756F069006D0E060031222E0900684
:10523200D4E060031223BC02553A900012E06006EB
:10524200A20DB3B34002801D900012E02529FFAEEB
:105252002850010E8E288F29E55DD39419500690AF
:105262000012E014F01212F1756F079006D8E06098
:10527200031224989006DCE0600312257402553A6A
:10528200900109E0B40203120CCD12154E756F089D
:105292009006E0E060031226509006E4E0600312FC
:1052A200272C02553A12190AA20D4015900017E058
:1052B200FEA3E0FF7402126530900017EEF0A3EF38
:1052C200F0A216B35005A217B340028006D216D23E
:1052D20017D218756F109006E8E060031228089044
:1052E20006ECE060031228E402553A02553A9000B7
:1052F20039E0C394465008C2967446900039F09043
:105302000049E0B4011DE534240CF5349007BDE0FA
:10531200FEA3E0FF740C2FFF50010E9007BDEEF0CC
:10532200A3EFF0900049E0B4021DE5342418F534EF
:105332009007BDE0FEA3E0FF74182FFF50010E900E
:1053420007BDEEF0A3EFF085345A75590090004383
:10535200E0F5721236B5E55C900039F0900006E592
:1053620059F0A3E55AF0E57290003AF0C21A90079C
:10537200BDE0F559A3E0F55A900043E0F57212360C
:10538200B5E55C900037F0900000E559F0A3E55ACE
:10539200F0E572900038F0C219E56CB40105756F42
:1053A2000B8003756F0302553A90003DE0C39446AB
:1053B20050139000D7E0B40104C2968002C29574E3
:1053C2004690003DF090004AE0B4011DE534240C03
:1053D200F5349007BDE0FEA3E0FF740C2FFF5001EF
:1053E2000E9007BDEEF0A3EFF090004AE0B4021D6C
:1053F200E5342418F5349007BDE0FEA3E0FF7418ED
:105402002FFF50010E9007BDEEF0A3EFF085345A46
:10541200755900900044E0F5721236B5E55C9000D3
:105422003DF0900008E559F0A3E55AF0E5729000CE
:105432003EF0C21C9007BDE0F559A3E0F55A90007A
:1054420044E0F5721236B5E55C90003BF090000244
:10545200E559F0A3E55AF0E57290003CF0C21BE575
:105462006CB40105756F0C8003756F0302553A9099
:105472000041E0C3944650139000D7E0B40104C247
:10548200968002C2A07446900041F090004BE0B4B6
:10549200011DE534240CF5349007BDE0FEA3E0FFC6
:1054A200740C2FFF50010E9007BDEEF0A3EFF090A9
:1054B200004BE0B4021DE5342418F5349007BDE03A
:1054C200FEA3E0FF74182FFF50010E9007BDEEF00F
:1054D200A3EFF085345A755900900045E0F5721239
:1054E20036B5E55C900041F090000AE559F0A3E57D
:1054F2005AF0E572900042F0C21E9007BDE0F559E5
:10550200A3E0F55A900045E0F5721236B5E55C90DD
:10551200003FF0900004E559F0A3E55AF0E57290DF
:105522000040F0C21DE56CB40103756C00756F0399
:08553200800680048002800065
:105DCA0002522102523C0252820252A70252ED02B0
:105DDA0052F00253AB025471025534025536025541
:045DEA003802553AEC
:10553A00900037E0B55D0280030255DCA219407283
:10554A00900000E0FEA3E0FFEF4E6021AE55AF569B
:10555A00900000E0FCA3E0FD120003740C8E048F9F
:10556A0005FF126520900000ECF0A3EDF0900038E2
:10557A00E0601A900000E0FEA3E0FFAC55AD56EFE4
:10558A002DFDEE3CFC900000ECF0A3EDF09000380D
:10559A00E0D39401401A900000E0FEA3E0FFAC556E
:1055AA00AD56EF2DFDEE3CFC900000ECF0A3EDF0C3
:1055BA00D219AE53AF54900000E0FCA3E0FDEFC354
:1055CA009DEE9C400D123F50D296C21974C89000AD
:1055DA0037F0A219B3B35007900037E0B55D0280E7
:1055EA000D123F50D29674C8900037F0C21990003D
:1055FA0039E0B55D028003025697A21A4072900004
:10560A0006E0FEA3E0FFEF4E6021AE55AF569000D4
:10561A0006E0FCA3E0FD120003740C8E048F05FF64
:10562A00126520900006ECF0A3EDF090003AE060DD
:10563A001A900006E0FEA3E0FFAC55AD56EF2DFD33
:10564A00EE3CFC900006ECF0A3EDF090003AE0D3BB
:10565A009401401A900006E0FEA3E0FFAC55AD5657
:10566A00EF2DFDEE3CFC900006ECF0A3EDF0D21A13
:10567A00AE53AF54900006E0FCA3E0FDEFC39DEEED
:10568A009C400AC2967446900039F0C21AA21AB314
:10569A00B35007900039E0B55D02800AC29674469D
:1056AA00900039F0C21A90003BE0B55D0280030217
:1056BA00575DA21B4072900002E0FEA3E0FFEF4E8E
:1056CA006021AE55AF56900002E0FCA3E0FD120047
:1056DA0003740C8E048F05FF126520900002ECF013
:1056EA00A3EDF090003CE0601A900002E0FEA3E017
:1056FA00FFAC55AD56EF2DFDEE3CFC900002ECF0F0
:10570A00A3EDF090003CE0D39401401A900002E02F
:10571A00FEA3E0FFAC55AD56EF2DFDEE3CFC90002C
:10572A0002ECF0A3EDF0D21BAE53AF54900002E0AE
:10573A00FCA3E0FDEFC39DEE9C4018123F50900081
:10574A00D7E0B40104D2968002D295C21B74C890E5
:10575A00003BF0A21BB3B3500790003BE0B55D02DB
:10576A008018123F509000D7E0B40104D29680020C
:10577A00D29574C890003BF0C21B90003DE0B55D25
:10578A0002800302582EA21C4072900008E0FEA379
:10579A00E0FFEF4E6021AE55AF56900008E0FCA343
:1057AA00E0FD120003740C8E048F05FF1265209031
:1057BA000008ECF0A3EDF090003EE0601A900008BB
:1057CA00E0FEA3E0FFAC55AD56EF2DFDEE3CFC909C
:1057DA000008ECF0A3EDF090003EE0D39401401AEB
:1057EA00900008E0FEA3E0FFAC55AD56EF2DFDEEAC
:1057FA003CFC900008ECF0A3EDF0D21CAE53AF5481
:10580A00900008E0FCA3E0FDEFC39DEE9C401590DC
:10581A0000D7E0B40104C2968002C2957446900093
:10582A003DF0C21CA21CB3B3500790003DE0B55D29
:10583A000280159000D7E0B40104C2968002C29596
:10584A00744690003DF0C21C90003FE0B55D0280B6
:10585A00030258FFA21D4072900004E0FEA3E0FF7D
:10586A00EF4E6021AE55AF56900004E0FCA3E0FD78
:10587A00120003740C8E048F05FF12652090000439
:10588A00ECF0A3EDF0900040E0601A900004E0FE16
:10589A00A3E0FFAC55AD56EF2DFDEE3CFC900004A5
:1058AA00ECF0A3EDF0900040E0D39401401A900090
:1058BA0004E0FEA3E0FFAC55AD56EF2DFDEE3CFC37
:1058CA00900004ECF0A3EDF0D21DAE53AF5490005B
:1058DA0004E0FCA3E0FDEFC39DEE9C4018123F508C
:1058EA009000D7E0B40104D2968002D2A0C21D74FF
:1058FA00C890003FF0A21DB3B3500790003FE0B537
:10590A005D028018123F509000D7E0B40104D2968D
:10591A008002D2A074C890003FF0C21D900041E0FE
:10592A00B55D0280030259D0A21E407290000AE0BF
:10593A00FEA3E0FFEF4E6021AE55AF5690000AE09D
:10594A00FCA3E0FD120003740C8E048F05FF1265A0
:10595A002090000AECF0A3EDF0900042E0601A906B
:10596A00000AE0FEA3E0FFAC55AD56EF2DFDEE3C7C
:10597A00FC90000AECF0A3EDF0900042E0D3940111
:10598A00401A90000AE0FEA3E0FFAC55AD56EF2D99
:10599A00FDEE3CFC90000AECF0A3EDF0D21EAE53F3
:1059AA00AF5490000AE0FCA3E0FDEFC39DEE9C40DB
:1059BA00159000D7E0B40104C2968002C2A07446D2
:1059CA00900041F0C21EA21EB3B35007900041E0FE
:1059DA00B55D0280159000D7E0B40104C29680023A
:1059EA00C2A07446900041F0C21E9000D9E0B402F1
:1059FA00028003025B10900073E0D39565506490B7
:105A0A000073E0F4042565FE9000DCE08E00F5F0FA
:105A1A00E884FF7E008F72EFC39410500CEF8572FA
:105A2A00F0A4FDACF08D7280037572FF900073E0F4
:105A3A00D39572400B900073E0C39572F5708003A2
:105A4A007570009000F7E0D3957040069000F7E07B
:105A5A00F5709000F8E0C3957050069000F8E0F5F4
:105A6A00708071900073E0C39565FE9000DCE08E53
:105A7A0000F5F0E884FF7E008F72EFC39410500C9B
:105A8A00EF8572F0A4FDACF08D7280037572FF850C
:105A9A00725A755900900073E0255AFFAE595001A9
:105AAA000E8E598F5A74FFBE0009D39F4005855A3E
:105ABA007080037570FF9000F7E0D39570400690F0
:105ACA0000F7E0F5709000F8E0C39570500690007A
:105ADA00F8E0F570A20DB3B3500D900074E0FE909B
:105AEA0000E4E0D39E5002800A7407900050F0C28E
:105AFA0097801375A710E5CDC395704004C29780AF
:105B0A0002D29775A700E56EC39409500AA2EDB3B5
:105B1A004005C2ED122C7AAE53AF547450C39F7431
:105B2A00469E400C900072E0C3945A4003025D8284
:105B3A00A213B34009123DDC7406900050F0A22172
:105B4A00B34008E5B54404F5B58006E5B554FBF560
:105B5A00B5A215B3500EE560D394334007E560C390
:105B6A0094CC4002802FE5B54401F5B5742390002A
:105B7A0071F0900085E075F0BEA4FFAEF08E5B8FE9
:105B8A005C7402BE000AD39F4006755C02755B0016
:105B9A00123EBCD215900072E0D394014007E56032
:105BAA00C3941A40028002C2159006C8E06003122C
:105BBA002114A22B300301B35017A22BB34008E5DE
:105BCA00B54408F5B58006E5B554F7F5B5A22B92AC
:105BDA00039006CCE060031221F0A22C300401B33A
:105BEA005017A22CB34008E5B54402F5B58006E586
:105BFA00B554FDF5B5A22C92049006D0E0600312CC
:105C0A0022E0A22D300501B3500FA22DB34004D2D9
:105C1A00978002C297A22D92059006D4E0600312E3
:105C2A0023BCA22E300601B3500FA22EB34004D2D9
:105C3A00A28002C2A2A22E92069006D8E0600312A7
:105C4A002498A22F300701B3500FA22FB34004D2D9
:105C5A00A18002C2A1A22F92079006DEE060031281
:105C6A002574A230300801B35017A230B34008E5BA
:105C7A00B54440F5B58006E5B554BFF5B5A23092F6
:105C8A00089006E0E06003122650A231300901B301
:105C9A005017A231B34008E5B54480F5B58006E552
:105CAA00B5547FF5B5A23192099006E4E06003127B
:105CBA00272CA232300A01B3500FA232B34004D2C9
:105CCA00928002C292A232920A9006E8E06003121F
:105CDA002808A233300B01B3500FA233B34004D2C9
:105CEA00878002C287A233920B9006ECE06003120F
:105CFA0028E4A234300C01B3500FA234B34004D2CA
:105D0A00908002C290A234920C900072E0C3945A1E
:105D1A005010E56EB40909900072E004F0756E0047
:105D2A00803BE56EB40903756E0075540075530027
:105D3A00758D00758B00756300900071E0C3943215
:105D4A005008900071E004F080067432900071F0FF
:105D5A00900071E0B43206E5B554FEF5B5900072D4
:105D6A00E0D394014007E569C39441400280097475
:0B5D7A000E900050F0123DDC02466667
:105E18000000010001400160018001A001C001E013
:105E280002000300039603B603D603F4040005003A
:105E38000512052405360548055A056C057E0590AA
:105E480005A805C005DE0600061406280646066EE7
:105E580006AE00FF013F015F017F019F01BF01DF27
:105E680001FF02FF039503B503D503F303FF04FF06
:105E780005110523053505470559056B057D058F72
:105E880005A705BF05DD05F1061306270645066DBE
:105E980006AD06ED0FAA0FA50F9F0F9A0F940F8D51
:105EA8000F870F800F780F710F680F600F570F4E15
:105EB8000F450F3B0F300F250F1A0F0E0F020EF56F
:105EC8000EE80EDB0ECC0EBE0EAE0E9F0E8E0E7DB5
:105ED8000E6C0E5A0E470E340E200E0C0DF70DE206
:105EE8000DCB0DB50D9D0D850D6D0D540D3A0D2085
:105EF8000D050CE90CCE0CB10C940C760C580C3A30
:105F08000C1B0BFB0BDB0BBB0B9A0B790B570B35E5
:105F18000B130AF10ACE0AAB0A870A640A400A1C64
:105F280009F809D409B0098C09670943091F08FB56
:105F380008D608B2088E086A0846082307FF07DC57
:105F480007B9079607730751072F070D06EC06CA0E
:105F580006AA068906690649062A060A05EC05CD39
:105F680005B0059205750558053C0520050504EAA8
:105F780004CF04B5049C0482046904510439042242
:105F8800040B03F403DE03C803B2039D03890375FE
:105F98000361034D033B03280316030402F202E1E5
:105FA80002D102C002B002A002910282027302650D
:105FB80002570249023C022F02220216020901FD81
:105FC80001F201E601DB01D001C601BB01B101A765
:105FD800019D0194018B01820179017001680160C2
:105FE800015801500148014101390132012B0125B5
:105FF800011E01180111010B010500FF00FA0FA68F
:106008000FA00F990F920F8B0F840F7C0F740F6BDB
:106018000F620F580F4E0F430F380F2C0F1F0F1220
:106028000F050EF70EE80ED80EC80EB70EA50E9384
:106038000E800E6C0E580E420E2C0E150DFD0DE442
:106048000DCB0DB10D950D790D5D0D3F0D200D0199
:106058000CE10CC00C9E0C7C0C590C350C100BEA96
:106068000BC40B9E0B760B4F0B260AFD0AD40AAA0B
:106078000A800A550A2A09FF09D409A8097C095087
:10608800092508F908CD08A10875084A081E07F36C
:1060980007C8079D07730749072006F706CE06A617
:1060A800067E06570630060A05E405BF059B0577F8
:1060B80005540532051004EF04CE04AE048F0471B4
:1060C80004530435041903FD03E203C703AD039425
:1060D800037B0363034B0334031E030802F302DE4E
:1060E80002CA02B602A30291027F026D025C024C50
:1060F800023C022C021D020E020001F201E401D74B
:1061080001CA01BE01B101A6019A018F0185017A78
:1061180001700166015D0153014A014101390131F4
:106128000129012101190112010B010400FD00F7E9
:1061380000F000EA00E400DE00D900D300CE00C978
:1061480000C400BF00BA00B500B100AD00A800A4AB
:1061580000A0009C009900950091008E008A00879D
:0861680000840081007E007B31
:10009E007547009007C5E4F0A3F075310075300088
:1000AE00754D00754E00C236D23774FE9007CFF8EC
:1000BE00E4F0E8A3F074FE9007D1F8E4F0E8A3F0C2
:1000CE00745A9007D3F0745A9007D4F0D238C22ADB
:1000DE00C23AC23522750B00750A00AE0AAF0BACE0
:1000EE0008AD09EDC39FEC9E401674FF12651075A6
:1000FE00CF01780B740126F6500418E436F650DB67
:10010E002290004CE0B4AA1C900781E0B43C1590FC
:10011E0007C1E0FEA3E0FFEF4E6009741EBE0004AF
:10012E00D39F500302023D755C00755B0075F809A4
:10013E009007C1E0FEA3E0FF74076F4E6006740ED9
:10014E006F4E7006743A900781F09007C1E0FEA3DF
:10015E00E0FF7408BE001ED39F401A7E017F0890F8
:10016E0007C1E0FCA3E0FD1DBDFF011C1200038EC4
:10017E00598F5A801F9007C1E0FEA3E0FF7408124A
:10018E0065748F048E057E017F08CDCCCD120003E1
:10019E008E598F5AAE5BAF5C740CD39F74019E5018
:1001AE0003020238A2F9B3407EE55C455B7003752D
:1001BE00A382AE5BAF5C74016F4E700375A300AE8D
:1001CE005BAF5C74026F4E700D9007C2E075F0026B
:1001DE00A4FDACF08DA3AE5BAF5C74036F4E7003E9
:1001EE0075A300AE5BAF5C7403BE00039F5013ACEF
:1001FE0059AD5AED2FFFEC3EFE90007D126557E093
:10020E00F5A3AE5BAF5CEFB40B09EEB4010574144D
:10021E00126510AE5BAF5CEFB40B07EEB401037565
:10022E00F80D785B1265840201A290004CE4F02276
:10023E00755C00755B0075F8099007C1E0FEA3E0E0
:10024E00FF7408BE001ED39F401A7E017F089007E0
:10025E00C1E0FCA3E0FD1DBDFF011C1200038E5981
:10026E008F5A801F9007C1E0FEA3E0FF740812654D
:10027E00748F048E057E017F08CDCCCD1200038EC7
:10028E00598F5AAE5BAF5C7411D39F74019E5003AD
:10029E0002036EA2F9B3500302036BE55C455B707B
:1002AE000375A3D2AE5BAF5C74016F4E700375A382
:1002BE0000AE5BAF5C74026F4E700D9007C2E075BE
:1002CE00F002A4FDACF08DA3AE5BAF5C74036F4E79
:1002DE00700375A300AE5BAF5C74046F4E70037554
:1002EE00A300AE5BAF5C74056F4E700375A300AEDA
:1002FE005BAF5C74066F4E700375A300AE5BAF5CB4
:10030E0074076F4E700375A300AE5BAF5C74086F1D
:10031E004E700375A300AE5BAF5C7408BE00039F06
:10032E005016AC59AD5AED2FFFEC3EFE90007812F0
:10033E006557E5A3F075A300AE5BAF5CEFB4100993
:10034E00EEB401057414126510AE5BAF5CEFB41021
:10035E0007EEB4010375F80D785B12658402029105
:10036E0022755C00755B0075F809AE5BAF5C7417A7
:10037E00BE0004D39F5003020447A2F9B3500302F8
:10038E000444E55C455B700375A3D2AE5BAF5C7451
:10039E00016F4E700375A300AE5BAF5C74026F4EBF
:1003AE00700D9007C2E075F002A4FDACF08DA3AE07
:1003BE005BAF5C74036F4E700375A300AE5BAF5CF6
:1003CE0074046F4E700375A300AE5BAF5C74056F63
:1003DE004E700375A300AE5BAF5C74066F4E700378
:1003EE0075A300AE5BAF5C74076F4E700375A30010
:1003FE00AE5BAF5C74086F4E700375A300AE5BAF5F
:10040E005C7408BE00039F500C90005A126557E5AD
:10041E00A3F075A300AE5BAF5C74166F4E700574DF
:10042E0014126510AE5BAF5C74166F4E700375F8E8
:10043E000D785B1265840203782290004CE0B4AB19
:10044E000280030204E2755C00755B0075F809AE6C
:10045E005BAF5C7412BE007CD39F4078A2F9B340B0
:10046E0070E55C455B700375A382AE5BAF5C740197
:10047E006F4E700375A300AE5BAF5C74026F4E706F
:10048E000D9007C2E075F002A4FDACF08DA3AE5B3B
:10049E00AF5C74036F4E700375A300AE5BAF5C74FC
:1004AE0003BE00039F500990005F126557E0F5A34D
:1004BE00AE5BAF5C74116F4E70057414126510AEA6
:1004CE005BAF5C74116F4E700375F80D785B12653F
:1004DE008402045D229007CCE4F074649007C1F8A6
:1004EE00E4F0E8A3F012036F74C89007C1F8E4F0CB
:1004FE00E8A3F0900066E0B4371A900063E0900035
:10050E005AF0900064E090005BF0900065E090007F
:10051E005CF080469007CC7401F074659007C1F8CA
:10052E00E4F0E8A3F012036F74C89007C1F8E4F08A
:10053E00E8A3F0900066E0B4371A900063E09000F4
:10054E005AF0900064E090005BF0900065E090003F
:10055E005CF0800674029007CCF09007CDE4F07446
:10056E00669007C1F8E4F0E8A3F012036F74C89028
:10057E0007C1F8E4F0E8A3F0900065E0B4371290FC
:10058E000063E0900054F0900064E090005DF08015
:10059E00769007CD7401F074679007C1F8E4F0E827
:1005AE00A3F012036F74C89007C1F8E4F0E8A3F04B
:1005BE00900065E0B43712900063E0900054F09024
:1005CE000064E090005DF0803E74029007CDF07400
:1005DE00689007C1F8E4F0E8A3F012036F74C890B6
:1005EE0007C1F8E4F0E8A3F0900065E0B43712908C
:1005FE000063E0900054F0900064E090005DF080A5
:10060E000674039007CDF022E54E64046006E5996A
:10061E0064FF6002802AA2364004D2368020E54E66
:10062E00600874E6254E900050F0754E00E54D6062
:10063E000874F0254D900050F0754D00C2368002C2
:10064E00C236E54E9033F8F8282873754E00E599BA
:10065E00B4FF03754D01E599B4FE03754D02E5999E
:10066E00B4FD03754D03E599B4FC03754D04E5998E
:10067E00B4FA03754D05E599B4FB06754E01123DAE
:10068E00DCE599B4F906754E04123DDCE599D39478
:10069E00E54007E599C394F04002801685994F75A1
:1006AE004E027E017F00E54FC394E61265308E3216
:1006BE008F339007C5E4F0A3F0E599D394C44007B7
:1006CE00E599C394E64002802885994F754E0374D0
:1006DE00E5C3954FF533753200AE32AF33905E18E9
:1006EE001264FFE493F87401939007C5C8F0A3C891
:1006FE00F0D299020AB3900063E070429007C5E011
:10070E00FEA3E0FF74FFBE00039F5009EFC39446A3
:10071E00EE940640119007C5E0FEA3E0FFEFD394E0
:10072E006DEE940640139007C5E0FEA3E0FF900027
:10073E0081126557E599F0800385997380119007B2
:10074E00C5E0FEA3E0FF900081126557E599F09099
:10075E0007C512653E9007C5E0FEA3E0FFEFB401AA
:10076E0006EEB40702800302089B900781E0B43CBA
:10077E00028003020885C29C900063E090011FF086
:10078E00900064E090008EF0900065E09000AEF076
:10079E00900066E09000D7F0900067E0900083F044
:1007AE00900068E09000C9F0900069E09000E7F0DA
:1007BE0090006AE09000BBF090006BE09000D9F0E2
:1007CE0090006CE0900109F012379A900075E0905D
:1007DE0000F0F0900076E09000A7F0900077E090A7
:1007EE0000A8F074639007C1F8E4F0E8A3F074ABCE
:1007FE0090004CF012044890004CE4F075096475BA
:10080E0008001200E3A2204038757201E572D394FD
:10081E0007502CE5729007C1F8E4F0E8A3F074AA33
:10082E0090004CF012010FE572C394075009750940
:10083E00647508001200E37872740126F650CD80BC
:10084E0036757208E572D3940E502CE5729007C17E
:10085E00F8E4F0E8A3F074AA90004CF012010FE552
:10086E0072C3940E50097509647508001200E3787E
:10087E0072740126F650CD74C89007C1F8E4F0E802
:10088E00A3F0D29C754E00754D007599FB020AB30C
:10089E009007C5E0FEA3E0FFEF4E70068599317517
:1008AE0030009007C5E0FEA3E0FF74016F4E701B91
:1008BE00AC30AD31AA32AB33ED2BFBEC3AFA8A06F3
:1008CE008B07900081126557E599F09007C5126568
:1008DE003E9007C5E0FEA3E0FF74026F4E7021ACA0
:1008EE0030AD3174566D4C7006E54F64E660028093
:1008FE0003123DDC12379A854F99754E00754D00E7
:10090E00020AB39007C5E0FEA3E0FF9000811265D6
:10091E0057E599F09007C512653E9007C5E0FEA316
:10092E00E0FFAC32AD338F028E038C068D07905EE6
:10093E005A1264FFE493F9740193FEEAD39EEB9985
:10094E004009854F99754E00754D00020AB3900708
:10095E00C5E0FEA3E0FF900081126557E599F09087
:10096E0007C512653E9007C5E0FEA3E0FFEFB40099
:10097E0006EEB401028003020AB390005CE075F04B
:10098E0002A4FDACF08D72ED900081126562EDFA5D
:10099E00E0FBEA900084126562EBFAE0FBEA2BFAC8
:1009AE0090005CE0B502028003020AA50DED9000F6
:1009BE0081126562E572FDE0FAED900085126562C6
:1009CE00EAFDE0FAEDC39AFD90005CE0B505028009
:1009DE0003020AA5E572900083126562E572FDE0DE
:1009EE00FAED900086126562EAFDE0FAED2AFD90BE
:1009FE00005CE0B505028003020AA5E5729000874F
:100A0E00126562FDE0FAED90005CE0F4042A9000BD
:100A1E0063F0E572900088126562FDE0FAED9000D9
:100A2E005CE0F4042A900064F0E57290008912658F
:100A3E0062FDE0FAED90005CE0F4042A900065F0AF
:100A4E00E57290008A126562FDE0FAED90005CE0BE
:100A5E00F4042A9007C1F8E4F0E8A3F074AB900018
:100A6E004CF01204487509647508001200E39007F3
:100A7E00C112653E1204487509647508001200E340
:100A8E009007C112653E1204487599F9750964758F
:100A9E0008001200E380FE7599FF75096475080061
:050AAE001200E380FED0
:0F33F80002065902070402089E02091102095C2D
:100AB30022E54D903407F8282873020B989007C558
:100AC300E0FEA3E0FF900052126557E0F59990070E
:100AD300C512653E9007C5E0FEA3E0FF74116F4E9B
:100AE3007003754D00020B98856D99020B98900762
:100AF300C5E0FEA3E0FF900081126557E0F599EF92
:100B0300B40107EEB40703754D009007C512653EA7
:070B1300020B989007C6E0F9
:0F340700020ABD020AC0020AEB020AF1020B160A
:100B1A009035BAF82828738552998067855E99803E
:100B2A0062856099805D856499805885669980534D
:100B3A00856799804E85689980498569998044902E
:100B4A00001AE0F599803CA237B340077599FAC2BA
:100B5A00378017A228B3400575990F800B90005073
:100B6A00E0F599900050E4F0C2288017856A9980D0
:100B7A0012856599800D856B9980087599FC8003AB
:030B8A00754D00A6
:1035BA00020B21020B26020B2B020B30020B3502E7
:1035CA000B3A020B3F020B44020B49020B51020B4E
:0D35DA0076020B7B020B80020B85020B8A30
:0B0B8D009007C512653E80031235E79B
:03341600020B9511
:100B980022E537255AFFAE5950010E9000811265A3
:100BA80057E0F538E537255AFFAE5950010E0FBF0B
:100BB80000010E900081126557E0F539853F3BE54D
:100BC80038B539058538378041E539D39538401D22
:100BD800E539C39538853AF0A4FFAEF0E53B8E04BD
:100BE8008F05FF126520ED2538F537801DE538C3E0
:100BF8009539853AF0A4FFAEF0E53B8E048F05FFEA
:100C0800126520EDF4042538F53722E539D39538F7
:100C1800401DE539C39538853AF0A4FFAEF0E53BB1
:100C28008E048F05FF126520ED2538F537801DE508
:100C380038C39539853AF0A4FFAEF0E53B8E048FB2
:100C480005FF126520EDF4042538F537229000875A
:100C5800E0B40170E56675F00A84FF7E008F37E521
:100C68006675F00A84ADF07C008D3A753F0A7559B7
:100C780005755A24E537C394115005120B9980065F
:100C88009005B6E0F537E53790007AF0E56675F03F
:100C98000A84FF7E008F37E56675F00A84ADF07C24
:100CA800008D3A753F0A755905755A5AE537C39448
:100CB800115005120B9980069005ECE0F537E537E1
:100CC800900012F022900087E0B4016AE56675F0A2
:100CD8000A84FF7E008F37E56675F00A84ADF07CE4
:100CE800008D3A753F0A755905755A36E537C3942C
:100CF800115005120B9980069005C8E0F537853725
:100D08004BE56675F00A84FF7E008F37E56675F05F
:100D18000A84ADF07C008D3A753F0A755905755AFD
:100D280048E537C394115005120B9980069005DAEF
:100D3800E0F53785374C22E55E75F00484FF7E00C8
:100D48008F37E55E75F00484ADF07C008D3A753F11
:100D580004755901755A00E537C3943F5005120BC5
:100D68009980069001C0E0F53785372975280090ED
:100D7800004FE075F020A4FFAEF09000D2E08E04A2
:100D88008F05FF1265208D379000BAE0D3955E502D
:100D980003020E459000DEE0D3955E4010ED900111
:100DA800C1126562E0F52B752A00020E429000A977
:100DB800E0D3955E4043E5379001C1126562E0F5E6
:100DC80038E5379001E1126562E0F5399000DEE020
:100DD800F404255EF53A9000A9E0FE9000DEE0F408
:100DE800042EF53BE538B539058538378003120CF4
:100DF8001385372B752A008041E5379001E112658C
:100E080062E0F538E537900201126562E0F5399045
:100E180000A9E0F404255EF53A9000BAE0FE9000DF
:100E2800A9E0F4042EF53BE538B539058538378057
:100E380003120C1385372B752A00020EEC9000E183
:100E4800E0D3955E5011E537900241126562E0F5F6
:100E58002B752A00020EEC9000AAE0D3955E504351
:100E6800E537900221126562E0F538E537900241D6
:100E7800126562E0F5399000AAE0F404255EF53ABF
:100E88009000E1E0FE9000AAE0F4042EF53BE5387E
:100E9800B539058538378003120C1385372B752A29
:100EA800008041E537900201126562E0F538E537C8
:100EB800900221126562E0F5399000BAE0F4042549
:100EC8005EF53A9000AAE0FE9000BAE0F4042EF530
:100ED8003BE538B539058538378003120C1385375B
:100EE8002B752A00229000F2E0F53C753F117559E8
:100EF80002755A00AE51AF52E53C75F00FA4FDAC37
:100F0800F0EDD39FEC9E4021E53C8E048F05FF1247
:100F18006520ED75F010A4FFAEF0E55E75F0118464
:100F2800FD7C00ED2FF53D800EE55E75F01184FF28
:100F38007E00EF24F0F53D853D37E55E75F01184C0
:100F4800AFF07E008F3A120B9985373EAE51AF5203
:100F58009000F2E075F00FA4FDACF0EDD39FEC9E8D
:100F68004028755902755A10853D37120B99853EF0
:100F780038853739AE51AF52E53C8E048F05FF12E4
:100F8800654B8D3A853C3B120C1385372975280033
:100F9800752B64752A00229000F2E0F53C753F112C
:100FA800755902755A00AE51AF52E53C75F00FA461
:100FB800FDACF0EDD39FEC9E4021E53C8E048F05FF
:100FC800FF126520ED75F010A4FFAEF0E56075F036
:100FD8001184FD7C00ED2FF53D800EE56075F01164
:100FE80084FF7E00EF24F0F53D853D37E56075F020
:100FF8001184AFF07E008F3A120B9985373EAE51BF
:10100800AF529000F2E075F00FA4FDACF0EDD39F65
:10101800EC9E4028755902755A10853D37120B9978
:10102800853E38853739AE51AF52E53C8E048F0581
:10103800FF12654B8D3A853C3B120C138537297599
:1010480028009000BCE0B40453E55E75F00484FF0A
:101058007E008F37E55E75F00484ADF07C008D3A34
:10106800753F04755901755A00E537C3943F50051B
:10107800120B9980069001C0E0F537AE28AF29E53C
:101088003712653074648E048F05FF126520AE2810
:10109800AF29EF2DFDEE3CFC8C288D29752B64754E
:1010A8002A0022900087E0B40146E56675F00A84BC
:1010B800FF7E008F37E56675F00A84ADF07C008D01
:1010C8003A753F0A755905755A00E537C3941150AA
:1010D80005120B998006900592E0F537AE2AAF2BE2
:1010E800E5372FFF50010E74641265748E2A8F2B1A
:1010F800900088E0B40146E56775F00A84FF7E0039
:101108008F37E56775F00A84ADF07C008D3A753F3E
:101118000A755905755A6CE537C394115005120BB9
:101128009980069005FEE0F537AE2AAF2BE5372FFC
:10113800FF50010E74641265748E2A8F2B900097ED
:10114800E0B40249E569C3944175F00584FF7E0067
:101158008F37E56975F00584ADF07C008D3A753FF1
:1011680005755906755A00E537C394135005120BD7
:10117800998006900694E0F537AE2AAF2BE5372F15
:10118800FF50010E74641265748E2A8F2B9000D95B
:10119800E0B40202800302124AE55E75F01584FF8E
:1011A8007E008F37E55E75F01584ADF07C008D3AD2
:1011B800753F15755903755AF4E537C3940B5005F7
:1011C800120B998006900480E0F537E53775F0FF3B
:1011D800A4FFAEF09000DAE08E048F05FF126520C0
:1011E800ED900073F0E56575F078A4FFAEF074FF3C
:1011F8008E048F05FF1265208C598D5A74028C0657
:101208008D071200398F37AC59AD5A7404FF126537
:101218004B8D3A753F04755906755A28E537C394BE
:101228001D5005120B9980069006C6E0F537AE2AC8
:10123800AF2BE5372FFF50010E74641265748E2AA8
:101248008F2B900086E0B4025DE56075F064A4FF22
:10125800AEF074081200398E5B8F5C74058E048FB3
:1012680005FF1265208D37AE5BAF5C74058E048F69
:1012780005FF12654B8D3A753F05755905755ADEA0
:10128800E537C394135005120B998006900672E057
:10129800F537AE2AAF2BE5372FFF50010E746412D5
:1012A80065748E2A8F2B9000C8E0703C90004FE048
:1012B80075F00584FF7E008F3790004FE075F005CC
:1012C80084ADF07C008D3A753F05755905755AC097
:1012D800E537C3941D5005120B99800690065EE011
:1012E800F537E53790007BF02290008FE0B40117C6
:1012F8009007C8E0252BFFAE2A50010E9000E3E0CE
:101308001265748E2A8F2B900107E0B401149001A6
:1013180008E0A851B8000495525007E55EC3955FF0
:10132800400280129000B1E0252BFFAE2A50010E3A
:101338008E2A8F2B802F90008FE0B40316A22AB339
:10134800B350109007CBE0C39405A851B800069598
:1013580052400280109000B1E0252BFFAE2A5001C8
:101368000E8E2A8F2B900089E0B4020280030215AA
:101378004D90008CE0602FE566D39446402890009D
:1013880013E0FEA3E0FF9000C7E075F003A4FDACF6
:10139800F0EFD39DEE9C400E9000EBE0A851B80012
:1013A80005D39552500302154D9000D4E0855EF0A8
:1013B800A4FFAEF0740512653074071200398E5917
:1013C8008F5A900093E0A851B8000495525012909B
:1013D8000094E075F002A4FDACF0EFC39DEE9C40D4
:1013E8000302154DE55E75F00B84FF7E0090061133
:1013F800126557FEE0FFEE90008BE0FEEF8E00884E
:10140800F0A4FFAEF074648E048F05FF1265208C83
:10141800598D5A90004FE075F018A4FFAEF0900077
:10142800D2E08E048F05FF1265208C068D0790068A
:1014380029126557AE59AF5AE012653074648E04AC
:101448008F05FF1265208C598D5AE564A859B8009C
:1014580077D3955A4072E564C3955AFFE49559FECF
:101468008E598F5A7428BE00039F500C755A2875E0
:101478005900740D900050F0AE59AF5A90008CE0AE
:1014880012653074288E048F05FF1265208C598DE3
:101498005AAE28AF29740A8E048F05FF1265208D75
:1014A800068C07AC59AD5ACFCECF120003740A8E02
:1014B800048F05FF1265208C598D5AAE28AF29126A
:1014C800657C8E288F29807DE564A859B80004952D
:1014D8005A5072AE59AF5AE5641265748E598F5AD4
:1014E8007428BE00039F500C755A28755900740D56
:1014F800900050F0AE59AF5A90008CE012653074ED
:10150800288E048F05FF1265208C598D5AAE28AF9E
:1015180029740A8E048F05FF1265208D068C07AC8E
:1015280059AD5ACFCECF120003740A8E048F05FF2F
:101538001265208C598D5AAE28AF29EF2DFDEE3C4F
:10154800FC8C288D29229000E7E0B4026AE55E75DC
:10155800F00884FF7E008F37E55E75F00884ADF0F3
:101568007C008D3A753F08755901755AE0E537C317
:10157800943F5005120B998006900280E0F537855C
:10158800372D752C00AE2CAF2DAC2AAD2B120003D5
:1015980074648E048F05FF1265208C2C8D2D9000AD
:1015A80084E08C068D0712653074648E048F05FF05
:1015B8001265208C2C8D2DAE28AF29AC2AAD2B12AC
:1015C800000374648E048F05FF1265208C288D2912
:1015D800900084E08C068D0712653074648E048F49
:1015E80005FF1265208C288D29A20D401DAE51AF34
:1015F800527405BE00039F5002D20DE560D394CC0F
:101608004008D2017411900050F09000E6E0B40256
:10161800089000E8E0640160028035AE28AF29E553
:101628006A12653074E78E048F05FF1265208C28D6
:101638008D299000E7E0B40217AE2CAF2DE56A12B1
:10164800653074E78E048F05FF1265208C2C8D2D74
:101658009000A6E05402601B90009DE0A851B800DD
:1016680012D39552400DA20DB3B35007E560C39451
:101678009A40028028AE35AF3690009BE075F002A4
:10168800A4FDACF0EF2DFDEE3CFC74022DFD5001E5
:101698000CE560BC0007D39D4003754301856036A7
:1016A800753500E54370030217919000F9E0C39582
:1016B800435003021783900109E0C394025076E572
:1016C8006675F00A84FF7E00900581126557E0F583
:1016D8005A755900AE59AF5A90009CE012653074A3
:1016E800648E048F05FF1265208C5B8D5C9000F979
:1016F800E004C395438C068D071265309000F9E02D
:101708008E048F05FF1265208C5B8D5CAE28AF2997
:10171800EF2DFDEE3CFC8C288D299000E7E0B4020B
:1017280012AE2CAF2DAA5BAB5CEF2BFBEE3AFA8A1C
:101738002C8B2D80469000F9E004C39543854BF02F
:10174800A4FFAEF09000F9E08E048F05FF1265202B
:101758008C5B8D5CAE28AF29EF2DFDEE3CFC8C2810
:101768008D299000E7E0B40212AE2CAF2DAA5BAB36
:101778005CEF2BFBEE3AFA8A2C8B2D05439000F98F
:10178800E0C3954350037543009000A6E054016000
:101798001B90009AE0A851B80012D39552400DA2B0
:1017A8000DB3B35007E55EC394CC4002802590008A
:1017B80098E075F003A4FFAEF0E5402FFF50010E4E
:1017C80074032FFF50010EE55EBE0007D39F400350
:1017D800754401855E40E54470030218C49000FA20
:1017E800E0C3954450030218B6900109E0C394027F
:1017F8005076E56675F00A84FF7E009005811265D3
:1018080057E0F55A755900AE59AF5A900099E01251
:10181800653074648E048F05FF1265208C5B8D5CC7
:101828009000FAE004C395448C068D071265309049
:1018380000FAE08E048F05FF1265208C5B8D5CAE8C
:1018480028AF29EF2DFDEE3CFC8C288D299000E770
:10185800E0B40212AE2CAF2DAA5BAB5CEF2BFBEE13
:101868003AFA8A2C8B2D80469000FAE004C39544FE
:10187800854CF0A4FFAEF09000FAE08E048F05FFCF
:101888001265208C5B8D5CAE28AF29EF2DFDEE3CF8
:10189800FC8C288D299000E7E0B40212AE2CAF2D05
:1018A800AA5BAB5CEF2BFBEE3AFA8A2C8B2D054436
:1018B8009000FAE0C3954450037544009000FCE0A2
:1018C8002529FFAE2850010E8E288F299000ABE005
:1018D800A828B80004952950099000ABE0F52975AF
:1018E80028009000E7E0B4020D9000ABE0A82CB807
:1018F8000006952D400280099000ABE0F52D752C6F
:1019080000229000E7E0B401028003021A15A20D3C
:10191800B35003021A139000B2E0B40168AE28AFC6
:1019280029AC51AD52120003743C8E048F05FF128E
:1019380065209000C2E0BC00109D400D9000C4E0FE
:10194800A828B8000495295002D202AE28AF29ACC5
:1019580051AD52120003743C8E048F05FF126520AE
:101968009000C2E0C3940ABC0015D39D40119000BA
:10197800C4E0C39405A828B80005D395295002806F
:1019880002C2028068AE28AF29AC51AD52120003E2
:1019980074788E048F05FF1265209000C2E0BC00A9
:1019A800109D400D9000C4E0A828B8000495295067
:1019B80004D2028038AE28AF29AC51AD52120003D0
:1019C80074788E048F05FF1265209000C2E0C394DE
:1019D8000ABC0015D39D40119000C4E0C39405A82B
:1019E80028B80005D3952950028002C202A202B38A
:1019F8004019AE28AF299000C3E012653074648E98
:101A0800048F05FF1265208C288D298002C202A24E
:101A180000B34006A201B3B35009900019E4F0A343
:101A2800F08024AE28AF297400D39F74019E400C27
:101A3800900019E528F0A3E529F0800B74FF9000C9
:101A480019F8E4F0E8A3F09000C9E0D39402400C40
:101A58009000B4E07006A20DB3B34002801AAE281D
:101A6800AF2974021265308E288F29AE2CAF2D74E1
:101A7800021265308E2C8F2D9000B2E0B4011AAEA0
:101A880028AF2974021265308E288F29AE2CAF2D0D
:101A980074021265308E2C8F2DAE28AF29745E1219
:101AA8006530740A8E048F05FF1265208C288D29F5
:101AB8009000E7E0B40217AE2CAF2D745E126530CB
:101AC800740A8E048F05FF1265208C2C8D2DAE288C
:101AD800AF297402BE000AD39F40067529027528F3
:101AE80000AE2CAF2D7402BE000AD39F4006752DA0
:101AF80002752C00900017E528F0A3E529F0229044
:101B0800004FE0900381126562E0F54175426490F0
:101B1800004FE0FE9000BDE0D39E4037E55E75F0D3
:101B28000884FF7E008F37E55E75F00884ADF07C91
:101B3800008D3A753F08755903755A96E537C39471
:101B48001F5005120B998006900436E0F53785374B
:101B5800428035E55E75F00884FF7E008F37E55ECC
:101B680075F00884ADF07C008D3A753F087559030F
:101B7800755AB6E537C3941F5005120B9980069025
:101B88000456E0F537853742229000F3E0F53C75BE
:101B98003F11755904755A00AE51AF52E53C75F0C6
:101BA8000FA4FDACF0EDD39FEC9E4021E53C8E04E4
:101BB8008F05FF126520ED75F010A4FFAEF0E55E0D
:101BC80075F01184FD7C00ED2FF53D800EE55E7506
:101BD800F01184FF7E00EF24F0F53D853D37E55E8A
:101BE80075F01184AFF07E008F3A120B9985373E5D
:101BF800AE51AF529000F3E075F00FA4FDACF0EDDC
:101C0800D39FEC9E4028755904755A10853D3712AC
:101C18000B99853E38853739AE51AF52E53C8E0475
:101C28008F05FF12654B8D3A853C3B120C138537A7
:101C380041754264229000F3E0F53C753F117559F7
:101C480004755A00AE51AF52E53C75F00FA4FDACD7
:101C5800F0EDD39FEC9E4021E53C8E048F05FF12EA
:101C68006520ED75F010A4FFAEF0E56075F0118405
:101C7800FD7C00ED2FF53D800EE56075F01184FFC9
:101C88007E00EF24F0F53D853D37E56075F0118461
:101C9800AFF07E008F3A120B9985373EAE51AF52A6
:101CA8009000F3E075F00FA4FDACF0EDD39FEC9E2F
:101CB8004028755904755A10853D37120B99853E91
:101CC80038853739AE51AF52E53C8E048F05FF1287
:101CD800654B8D3A853C3B120C1385374175426440
:101CE8009000EEE0B4047990004FE0FE9000BDE073
:101CF800D39E4037E55E75F00884FF7E008F37E598
:101D08005E75F00884ADF07C008D3A753F08755912
:101D180003755A96E537C3941F5005120B99800630
:101D2800900436E0F5378537428035E55E75F00872
:101D380084FF7E008F37E55E75F00884ADF07C0087
:101D48008D3A753F08755903755AB6E537C3941F20
:101D58005005120B998006900456E0F537853742F6
:101D680022900087E0B4013BE56675F00A84FF7EA7
:101D7800008F37E56675F00A84ADF07C008D3A7502
:101D88003F0A755905755A12E537C3941150051263
:101D98000B9980069005A4E0F537E5422537C394F2
:101DA80064F542900088E0B4013BE56775F00A8469
:101DB800FF7E008F37E56775F00A84ADF07C008DF3
:101DC8003A753F0A755905755A7EE537C39411501F
:101DD80005120B998006900610E0F537E542253785
:101DE800C39464F542E5412542F53490008FE0B490
:101DF80002109007C7E02534FE9000E3E0F4042EBB
:101E0800F5349000E6E0D394014040E56AC394E7D6
:101E1800501D74E7C3956AFE9007C9E08E00F5F07F
:101E2800E884FF7E008F37E5342537F534801CE5DC
:101E38006AC394E7FE9007C9E08E00F5F0E884FFD6
:101E48007E008F37E534C39537F534A20D4006E59B
:101E5800412464F534E534D394644009E534C394EB
:101E680064F53480037534009000BFE0C3953450A6
:101E7800069000BFE0F53422D200900079E0A85126
:101E8800B8000495525041900079E0A851B8000478
:101E98009552500375340F900079E004A851B800AA
:101EA800049552500375340A900079E02402A85131
:101EB800B8000495525005753405C200900079E0C9
:101EC80060067409900050F0C23A7E017F009000CD
:101ED800C5E01265309000D4E08E048F05FF1265CE
:101EE80020E55EBC0017D39D40139000CEE0B402FD
:101EF80004D23A8002C200740A900050F09000C6E2
:101F0800E0C3956650159000D8E0A851B800049534
:101F1800525002C200740B900050F0E566C39464FE
:101F2800501D90011EE0600D90011EE0A851B80000
:101F380006955240028008C200740B900050F0A22F
:101F4800004003753405900107E0B40114900108BE
:101F5800E0A851B8000495525007E55EC3955F406C
:101F68000280089000B0E0F534803A90008FE0B429
:101F78000306A22AB3B34002802B9007CBE0C39498
:101F880005A851B800049552500C9000B0E0F53403
:101F9800740C900050F09007CBE0A851B80004955D
:101FA800525002C20085346B900081E02534FE90C7
:101FB800004FE075F01E84FC7F00EE2CF534229073
:101FC800004FE075F00584FF7E008F3790004FE0EA
:101FD80075F00584ADF07C008D3A753F05755903A1
:101FE800755AD69000D2E01475F00584FF7E00E59E
:101FF80037BE00039F5005120B99800BE5379004FC
:1020080057126562E0F537E5379007CAF09007CABE
:10201800E0FE9000C1E0C39E50089000C1E0900728
:10202800CAF022E56675F00A84FF7E0090058112E9
:102038006557E0F546E546D394644010E546C394F9
:102048006475F00F84FF7E008F468003754600900C
:1020580000A4E02546F546229007BBE0FEA3E0FF7A
:102068007404120039E55E126530740F8E048F0512
:10207800FF1265209007B9ECF0A3EDF0900097E00F
:10208800B40262E569C3944175F00584FF7E008F50
:1020980037E56975F00584ADF07C008D3A753F052C
:1020A800755906755A14E537C394175005120B99DC
:1020B80080069006A8E0F5379007B9E0FEA3E0FF98
:1020C800740A8E048F05FF126520E5378C068D078C
:1020D800126530740A8E048F05FF1265209007B9C7
:1020E800ECF0A3EDF09007B9E0FEA3E0FF9007BF86
:1020F800E0FCA3E0FDEDD39FEC9E400F9007BFE00E
:10210800F8A3E09007B9C8F0A3C8F0229006C8E089
:10211800903419F8282873804C85527280479000B3
:10212800D4E0855EF0A4FFAEF074081200398F7217
:102138008033856072802E856672802985677280FB
:1021480024856872801F856972801A856A72801575
:102158008565728010856472800B856B728006902D
:05216800001AE0F57211
:1034190002211F02212102212602213A02213F0213
:10342900214402214902214E02215302215802213D
:073439005D02216202216720
:10216D009006C9E0FE9006CAE0D39E404B9006C88B
:10217D00E0B404189006CAE0C395725002D22B90B9
:10218D0006C9E0D395724002C22B802A9006C9E0A1
:10219D00C3957250099006CAE0D395725002800221
:1021AD00D22B9006C9E0D3957250099006CAE0C3B0
:1021BD0095725002C22B802A9006C9E0D3957240C9
:1021CD00099006CAE0C3957240028002C22B9006A8
:1021DD00C9E0C3957240099006CAE0D395724002DA
:1021ED00D22B229006CCE0903440F8282873804CF6
:1021FD0085527280479000D4E0855EF0A4FFAEF06A
:10220D0074081200398F728033856072802E856656
:10221D007280298567728024856872801F85697236
:10222D00801A856A7280158565728010856472804A
:0C223D000B856B72800690001AE0F572B1
:103440000221FB0221FD02220202221602221B029D
:10345000222002222502222A02222F0222340222C4
:073460003902223E02224363
:102249009006CDE0FE9006CEE0D39E405F9006CC8E
:10225900E0B404189006CEE0C395725002D22C90D7
:1022690006CDE0D395724002C22C803E9006CDE0A7
:10227900C3957250099006CEE0D395725002800240
:10228900D22C9006CDE0D3957250099006CEE0C3CA
:1022990095725002C22C9006CCE0B401099000E07E
:1022A900E0D3956050028002C22C802A9006CDE0CE
:1022B900D3957240099006CEE0C395724002800220
:1022C900C22C9006CDE0C3957240099006CEE0D3AA
:1022D90095724002D22C229006D0E0903467F828FB
:1022E9002873804C85527280479000D4E0855EF057
:1022F900A4FFAEF074081200398F728033856072C2
:10230900802E85667280298567728024856872802F
:102319001F856972801A856A7280158565728010B9
:10232900856472800B856B72800690001AE0F572E5
:103467000222EB0222ED0222F202230602230B02C2
:10347700231002231502231A02231F0223240223E7
:073487002902232E0223336A
:102339009006D1E0FE9006D2E0D39E404B9006D0A5
:10234900E0B404189006D2E0C395725002D22D90E1
:1023590006D1E0D395724002C22D802A9006D1E0C1
:10236900C3957250099006D2E0D39572500280024B
:10237900D22D9006D1E0D3957250099006D2E0C3D0
:1023890095725002C22D802A9006D1E0D3957240F1
:10239900099006D2E0C3957240028002C22D9006D0
:1023A900D1E0C3957240099006D2E0D395724002FC
:1023B900D22D229006D4E090348EF8282873804CD0
:1023C90085527280479000D4E0855EF0A4FFAEF09C
:1023D90074081200398F728033856072802E856689
:1023E9007280298567728024856872801F85697269
:1023F900801A856A7280158565728010856472807D
:0C2409000B856B72800690001AE0F572E3
:10348E000223C70223C90223CE0223E20223E7024C
:10349E0023EC0223F10223F60223FB022400022472
:0734AE000502240A02240FAD
:102415009006D5E0FE9006D6E0D39E404B9006D4BC
:10242500E0B404189006D6E0C395725002D22E90FF
:1024350006D5E0D395724002C22E802A9006D5E0DB
:10244500C3957250099006D6E0D39572500280026A
:10245500D22E9006D5E0D3957250099006D6E0C3EA
:1024650095725002C22E802A9006D5E0D39572400F
:10247500099006D6E0C3957240028002C22E9006EE
:10248500D5E0C3957240099006D6E0D39572400217
:10249500D22E229006D8E09034B5F8282873804CC7
:1024A50085527280479000D4E0855EF0A4FFAEF0BF
:1024B50074081200398F728033856072802E8566AC
:1024C5007280298567728024856872801F8569728C
:1024D500801A856A728015856572801085647280A0
:0C24E5000B856B72800690001AE0F57207
:1034B5000224A30224A50224AA0224BE0224C302D4
:1034C50024C80224CD0224D20224D70224DC0224FB
:0734D500E10224E60224EBF2
:1024F1009006D9E0FE9006DAE0D39E404B9006D8D4
:10250100E0B404189006DAE0C395725002D22F901D
:1025110006D9E0D395724002C22F802A9006D9E0F5
:10252100C3957250099006DAE0D395725002800289
:10253100D22F9006D9E0D3957250099006DAE0C304
:1025410095725002C22F802A9006D9E0D39572402D
:10255100099006DAE0C3957240028002C22F90060C
:10256100D9E0C3957240099006DAE0D39572400232
:10257100D22F229006DCE09034DCF8282873804CBE
:1025810085527280479000D4E0855EF0A4FFAEF0E2
:1025910074081200398F728033856072802E8566CF
:1025A1007280298567728024856872801F856972AF
:1025B100801A856A728015856572801085647280C3
:0C25C1000B856B72800690001AE0F5722A
:1034DC0002257F02258102258602259A02259F025C
:1034EC0025A40225A90225AE0225B30225B8022582
:0734FC00BD0225C20225C735
:1025CD009006DDE0FE9006DEE0D39E404B9006DCEB
:1025DD00E0B404189006DEE0C395725002D230903C
:1025ED0006DDE0D395724002C230802A9006DDE010
:1025FD00C3957250099006DEE0D3957250028002A9
:10260D00D2309006DDE0D3957250099006DEE0C31E
:10261D0095725002C230802A9006DDE0D39572404B
:10262D00099006DEE0C3957240028002C23090062A
:10263D00DDE0C3957240099006DEE0D3957240024D
:10264D00D230229006E0E0903503F8282873804CB4
:10265D0085527280479000D4E0855EF0A4FFAEF005
:10266D0074081200398F728033856072802E8566F2
:10267D007280298567728024856872801F856972D2
:10268D00801A856A728015856572801085647280E6
:0C269D000B856B72800690001AE0F5724D
:1035030002265B02265D02266202267602267B02E3
:10351300268002268502268A02268F022694022608
:073523009902269E0226A377
:1026A9009006E1E0FE9006E2E0D39E404B9006E002
:1026B900E0B404189006E2E0C395725002D231905A
:1026C90006E1E0D395724002C231802A9006E1E02A
:1026D900C3957250099006E2E0D3957250028002C8
:1026E900D2319006E1E0D3957250099006E2E0C339
:1026F90095725002C231802A9006E1E0D39572406A
:10270900099006E2E0C3957240028002C231900648
:10271900E1E0C3957240099006E2E0D39572400268
:10272900D231229006E4E090352AF8282873804CAB
:1027390085527280479000D4E0855EF0A4FFAEF028
:1027490074081200398F728033856072802E856615
:102759007280298567728024856872801F856972F5
:10276900801A856A72801585657280108564728009
:0C2779000B856B72800690001AE0F57270
:10352A0002273702273902273E022752022757026B
:10353A00275C02276102276602276B02277002278F
:07354A007502277A02277FBA
:102785009006E5E0FE9006E6E0D39E404B9006E419
:10279500E0B404189006E6E0C395725002D2329078
:1027A50006E5E0D395724002C232802A9006E5E044
:1027B500C3957250099006E6E0D3957250028002E7
:1027C500D2329006E5E0D3957250099006E6E0C353
:1027D50095725002C232802A9006E5E0D395724088
:1027E500099006E6E0C3957240028002C232900667
:1027F500E5E0C3957240099006E6E0D39572400284
:10280500D232229006E8E0903551F8282873804CA2
:1028150085527280479000D4E0855EF0A4FFAEF04B
:1028250074081200398F728033856072802E856638
:102835007280298567728024856872801F85697218
:10284500801A856A7280158565728010856472802C
:0C2855000B856B72800690001AE0F57293
:1035510002281302281502281A02282E02283302F3
:10356100283802283D02284202284702284C022816
:073571005102285602285BFD
:102861009006E9E0FE9006EAE0D39E404B9006E830
:10287100E0B404189006EAE0C395725002D2339096
:1028810006E9E0D395724002C233802A9006E9E05E
:10289100C3957250099006EAE0D395725002800206
:1028A100D2339006E9E0D3957250099006EAE0C36D
:1028B10095725002C233802A9006E9E0D3957240A6
:1028C100099006EAE0C3957240028002C233900685
:1028D100E9E0C3957240099006EAE0D3957240029F
:1028E100D233229006ECE0903578F8282873804C9A
:1028F10085527280479000D4E0855EF0A4FFAEF06F
:1029010074081200398F728033856072802E85665B
:102911007280298567728024856872801F8569723B
:10292100801A856A7280158565728010856472804F
:0C2931000B856B72800690001AE0F572B6
:103578000228EF0228F10228F602290A02290F027E
:10358800291402291902291E02292302292802299D
:073598002D02293202293740
:10293D009006EDE0FE9006EEE0D39E404B9006EC47
:10294D00E0B404189006EEE0C395725002D23490B4
:10295D0006EDE0D395724002C234802A9006EDE078
:10296D00C3957250099006EEE0D395725002800225
:10297D00D2349006EDE0D3957250099006EEE0C387
:10298D0095725002C234802A9006EDE0D3957240C4
:10299D00099006EEE0C3957240028002C2349006A3
:1029AD00EDE0C3957240099006EEE0D395724002BA
:1029BD00D23422AE2EAF2F74F5D39F74019E4008F2
:1029CD00782E126584022ADA752F01752E00AE510C
:1029DD00AF52E546BE000DD39F40099000B6E0D33F
:1029ED00954740028023754700E546C39552F57221
:1029FD009000B9E0D395454008E5452572F5458031
:102A0D00069000B9E0F54580020547900092E0D3AD
:102A1D009560401CE55EC3955F4015AE51AF52E524
:102A2D0046BE00039F50099000B7E0D39548400281
:102A3D00806E9007CEE0A851B800049552500375F2
:102A4D004A009007CEE0A851B8000BD3955240062E
:102A5D00E5529007CEF0E54A7041E552C39546F533
:102A6D0072E572D3940540037572059000B8E0C30A
:102A7D0095455007E572C3954540028009E545C36C
:102A8D009572F54580069000B8E0F5459000B8E0E8
:102A9D00D3954540069000B8E0F545754800800295
:102AAD000548E54A7016900092E0C39560500DE51B
:102ABD00462405A851B8000695524002800F90009B
:102ACD00A5E0F545754A0174789007CEF022AE2E3B
:102ADD00AF2F74E9D39F74039E4008782E1265843E
:102AED00022C79752F01752E00754532A235402ABD
:102AFD007545199000A5E075F002A4FFAEF0E5470D
:102B0D00BE0006D39F4002D2350547754A0374783F
:102B1D009007CEF0754900022C68AE51AF52E546D4
:102B2D006F4E7003022C68E546BE000DD39F400921
:102B3D009000B6E0D395474002800F754700E54AF7
:102B4D00C394035003754519800DE546C39552F5A1
:102B5D0072E5472572F547900092E0D39560400EDF
:102B6D009007CEE0A851B80007D395524002800CD3
:102B7D0005499000A5E0B54903754A00E54AB4033F
:102B8D0006A20DB3B34002800A0549E549B43C03E2
:102B9D00754A02E54AB402299007CEE0A851B80063
:102BAD000ED395524009E5529007CEF0754900902D
:102BBD000092E0C39560500975490074789007CE76
:102BCD00F0E54A705A900092E0D39560401CE55EA6
:102BDD00C3955F4015AE51AF52E546BE00039F5001
:102BED00099000B7E0D395484002800875480075FC
:102BFD00454B8028E552C39546F572E572D3940591
:102C0D004003757205900092E0D395604008E54849
:102C1D002572F5488006E5482406F548754900E516
:102C2D004A7016900092E0C39560500DE54624055C
:102C3D00A851B80006955240028003754A01E54A35
:102C4D00B4011875451905499000A5E0B5490675FB
:102C5D004A0275490074789007CEF0E54575F00A83
:102C6D00A4FFAEF09007C3EEF0A3EFF022E56E9057
:102C7D00359FF828287390008AE07003022E289063
:102C8D0000C0E0B401028003022D7890004DE0B544
:102C9D005D028003022D757E017F00E5BE12653059
:102CAD00E5BD2FFF50010E8E598F5A7410126530ED
:102CBD00900078E08E048F05FF1265209007CFEC11
:102CCD00F0A3EDF0E56A60089000E6E064026002B2
:102CDD0080269000E8E0B4011F9007CFE0FEA3E04E
:102CED00FF74E7126530E56A8E048F05FF126520CB
:102CFD009007CFECF0A3EDF090008AE0B40227909E
:102D0D0007D1E0FEA3E0FF9007CFE0FCA3E0FDEFCD
:102D1D002DFDEE3CFC74018C068D071200399007D9
:102D2D00CFEEF0A3EFF09007CFE0FEA3E0FF90070A
:102D3D00D1E0FCA3E0FDEDD39FEC9E4004D23880A2
:102D4D0002B2389007CFE0F8A3E09007D1C8F0A306
:102D5D00C8F09000BCE064016006A238B3B3400235
:102D6D0080069007D0E0F55E022E26D2387E017FD8
:102D7D0000E5BE126530E5BD2FFF50010E8E598F57
:102D8D005A7410126530900078E08E048F05FF1292
:102D9D0065209007CFECF0A3EDF0E56A6008900098
:102DAD00E6E06402600280269000E8E0B4011F9026
:102DBD0007CFE0FEA3E0FF74E7126530E56A8E04ED
:102DCD008F05FF1265209007CFECF0A3EDF090007A
:102DDD008AE0B402279007D1E0FEA3E0FF9007CF71
:102DED00E0FCA3E0FDEF2DFDEE3CFC74018C068DA7
:102DFD00071200399007CFEEF0A3EFF09007CFE068
:102E0D00F8A3E09007D1C8F0A3C8F09000BCE0642F
:102E1D000160069007D0E0F55E8003755E009000BE
:102E2D0086E07006756E01022C7A75BB180233F3BD
:102E3D00900086E07003022FC97E017F00E5BE126F
:102E4D006530E5BD2FFF50010E8E598F5A9000CC85
:102E5D00E0B4010F7E0F7FFFAC59AD5A12657C8E29
:102E6D00598F5A9000F1E0B40245AE59AF5A900017
:102E7D0023E0FCA3E0FDEDD39FEC9E400A900023E0
:102E8D00E559F0A3E55AF0AE59AF5A900025E0FC94
:102E9D00A3E0FDEFD39DEE9C400A900025E559F08F
:102EAD00A3E55AF0AE59AF5A74041200398F6090F1
:102EBD0000F1E0704CAE59AF5A900023E0FCA3E056
:102ECD00FDEFD39DEE9C400912657C8E598F5A8083
:102EDD0006755A00755900AE59AF5A741012653007
:102EED00900075E08E048F05FF1265208C598D5A68
:102EFD0074FFBC0009D39D4005855A608003756041
:102F0D00FE9000BCE0B401028003022FC7A20DB3F6
:102F1D00B3500E900090E0A851B80005D3955250D3
:102F2D0003022FBC900091E075F019A4FFAEF09054
:102F3D0000D4E08E048F05FF1265209000CDE08552
:102F4D0060F0A4FFAEF074648D028C038E048F05C7
:102F5D00FF126520EA2DFDEB3CFC8C598D5AE56A7C
:102F6D00600F9000E6E0B402089000E8E0640160B4
:102F7D00028017AE59AF5A74E7126530E56A8E04B8
:102F8D008F05FF1265208C598D5AAE59AF5A900797
:102F9D00CFE0FCA3E0FDEDD39FEC9E4005855A5E8E
:102FAD00800BA238B340069007D0E0F55E800BA2EF
:102FBD0038B340069007D0E0F55E80037560009051
:102FCD000089E07006756E02022C7A75BB1902330A
:102FDD00F3900089E0700302307EE55DD39550409B
:102FED000302307C900021E0FEA3E0FFE564126552
:102FFD0074900021EEF0A3EFF07E017F00E5BE128C
:10300D006530E5BD2FFF50010E8E598F5A9000F699
:10301D00E07013740A12653074518E048F05FF121F
:10302D0065208D648019AE59AF5A740A1265308FC0
:10303D00048E057E017F95CDCCCD12641E8F64E587
:10304D0064D394644003756464900021E0FEA3E0B2
:10305D00FFE5642FFF50010E900021EEF0A3EFF07D
:10306D0090008DE0048E048F05FF1265208D648025
:10307D00037564329000D9E07006756E03022C7AE8
:10308D0075BB130233F39000D9E0604A7E017F00D7
:10309D00E5BE126530E5BD2FFF50010E8E598F5ADA
:1030AD0074041200398F659000DBE08565F0A4FD96
:1030BD00ACF07464FF1265208D659000DAE08565D3
:1030CD00F0A4FFAEF074FF8E048F05FF126520EDA6
:1030DD00900074F08003756500900087E0700675B0
:1030ED006E04022C7A75BB170233F3900087E0B49F
:1030FD000102800302318C7E017F00E5BE12653036
:10310D00E5BD2FFF50010E8E598F5A9007D3E06009
:10311D00199007D3E014905E9C12008CE493FC741C
:10312D000193FDEDC39FEC9E400280069007D3E016
:10313D0014F09007D3E0C394B3501DAE59AF5A901D
:10314D0007D3E004905E9C12008CE493FC74019311
:10315D00FDEFC39DEE9C400280069007D3E004F086
:10316D009007D3E0FE9000ADE08E0088F0A4FFAE96
:10317D00F074648E048F05FF1265208D66800375D3
:10318D006600900088E07006756E05022C7A75BB9E
:10319D00160233F3900088E0B40102800302323549
:1031AD007E017F00E5BE126530E5BD2FFF50010E9B
:1031BD008E598F5A9007D4E060199007D4E014907F
:1031CD00600612008CE493FC740193FDEDC39FEC3B
:1031DD009E400280069007D4E014F09007D4E0C31F
:1031ED0094B3501DAE59AF5A9007D4E004906006C9
:1031FD0012008CE493FC740193FDEFC39DEE9C4093
:10320D000280069007D4E004F09007D4E0FE900011
:10321D00B3E08E0088F0A4FFAEF074648E048F05C9
:10322D00FF1265208D67800375670075BB1F023324
:10323D00F37E017F00E5BE126530E5BD2FFF500125
:10324D000E8E598F5A740912653074E68E048F05EF
:10325D00FF1265208D6990008FE07006756E070274
:10326D002C7A75BB150233F390008FE07003023397
:10327D008F7E017F00E5BE126530E5BD2FFF500149
:10328D000E8E598F5A74041200398F6890008FE09A
:10329D00B401159000E3E08568F0A4FFAEF074076B
:1032AD00120039EF9007C8F090008FE0B40215902E
:1032BD0000E3E08568F0A4FFAEF07407120039EF6B
:1032CD009007C7F090008FE0B40302800302338DA6
:1032DD009000D0E070389000E3E0601CE568C39486
:1032ED00195002D22AE568D394644002C22A900094
:1032FD00AFE09007CBF08014E568C394195002D26B
:10330D0039E568D394324002C239C22A80639000F5
:10331D00AFE070349000E3E08568F0A4FFAEF07488
:10332D00FF8E048F05FF126520ED9007CBF0AE5197
:10333D00AF52741EBE0006D39F4002D22AE560D361
:10334D0094E54002C22A8029E568C3940A500DAE67
:10335D0051AF52741EBE0004D39F50028002D22A78
:10336D00E560D394E54002C22A9000AFE09007CB10
:10337D00F09007CBE0C39405500674059007CBF091
:10338D0080037568009000E6E07006756E08022CEB
:10339D007A75BB1480509000E6E060397E017F00A5
:1033AD00E5BE126530E5BD2FFF50010E8E598F5AC7
:1033BD00EFD39421EE940E4005756AFF8015AE593A
:1033CD00AF5A741012653074E38E048F05FF1265C9
:1033DD00208D6A8003756A0090008AE0600575BBD8
:0633ED001A800375BB18F5
:10359F00022C83022E3D022FDE0230930230F802FE
:0B35AF0031A102323E0232750233A34C
:0533F300056ED2EC2282
:096562002582F582500205832216
:0F008C0025E050020583258250020583F582226C
:1064FF00EF2F500205832582F582E5833E2EF5832B
:01650F002269
:10657400CFC39FFF50011E22C3EF9DFFEE9CFE225E
:086584000806B6000218062209
:0D653E00A3E004F07006120049E004F02212
:0E003900048007C3CE13CECF13CFD5E0F6223E
:10641E00BC000FBE0008ED8FF084FFADF022E4FE4D
:10642E00FF22BE000DEF60FE54F0606F20E7030206
:10643E0064D4EAC0E0EBC0E078017A0075F001EEBA
:10644E0020E710EF25E0FFEE33FE0AC5F023C5F07E
:10645E0030E7F0EA5407F9096A7A007B0060010818
:10646E00C3EC9E40167004ED9F4010ED9FFDEC9E18
:10647E00FCE5F0CA4ACA03F5F08005E5F003F5F035
:10648E00C3EE13FEEF13FFD9D77908CACBCAD8D003
:10649E00EAFEEBFFD0E0FBD0E0FA22EC8FF084FCBA
:1064AE00ED54F045F0C48FF084FEEDC454F045F089
:1064BE00C48FF084FDEEC4FE54F02DFFEE540F3C5D
:1064CE00FEADF07C0022790078008FF0EC7E082083
:1064DE00E70DC3CD33CD33C933C9C833C8DEF0841D
:1064EE0049F9E5F08FF0BE00E6FD7C00E9FFE8FE1D
:0164FE00227B
:0E653000F88FF0A4FFE5F0CE88F0A42EFE2236
:10000300EF8DF0A4F9A8F0EF8CF0A428F8EE8DF0B2
:06001300A428FEE9FF2213
:10651000600D782B02651A007830D8FED5E0F8229D
:10652000EEC0E07E0012641EEFFDEEFCD0E0FE2225
:0C654B00EEC0E07E0012641ED0E0FE22D4
:03001B0002001EC2
:0300530002005652
:03009B00020071EF
:0300000002656B2B
:09656B0075817475D00002400630
:0B655700E5822FF582E5833EF58322EC
:0A0049000582D5820215831582227C
:10001E00C0E0C0F0C083C082C0D075D000123F8552
:0B002E00D0D0D082D083D0F0D0E032E0
:10005600C0E0C0F0C083C082C0D075D000123F8817
:10006600D0D0D082D083D0F0D0E032C0E0C0F0C093
:1000760083C082C0D075D000123FA4D0D0D082D029
:0600860083D0F0D0E0324F
:00000001FF
